:020000040010EA
:20000000060000EAFEFFFFEAFEFFFFEAFEFFFFEAFEFFFFEAFEFFFFEAFEFFFFEAFEFFFFEAA6
:200020008109A0E3D3F021E300D0A0E114009FE50FE0A0E110FF2FE10C009FE50FE0A0E174
:2000400010FF2FE1FEFFFFEA3801100050001000000000EB6A0100EB2C008FE2000C90E890
:2000600000A08AE000B08BE001704AE20B005AE10000001A620100EB0F00BAE818E04FE236
:20008000010013E303F0471013FF2FE15008000080080000102052E27800B0287800A12828
:2000A000FBFFFF8A822EB0E13000B0283000A12800409045004081451EFF2FE10030B0E370
:2000C0000040B0E30050B0E30060B0E3102052E27800A128FCFFFF8A822EB0E13000A12814
:2000E000003081451EFF2FE17847C04604309FE503308FE013FF2FE1910700000000A0E183
:20010000FEFFFFEA1EFF2FE13F402DE900E0A0E101C0A0E10240A0E10350A0E1010B4CE2C3
:2001200000008DE504C08DE50F009DE810D08DE23040BDE81EFF2FE184009FE50219A0E34C
:200140000020A0E3BC1202E5301090E5031001E2030051E30000001A1EFF2FE164109FE526
:200160000020A0E3A01002E55C109FE5201080E50000A0E1681090E5010011E3FCFFFF0A59
:2001800048109FE52C1080E50000A0E1681090E5040011E3FCFFFF0A0000A0E1681090E50A
:2001A000080011E3FCFFFF0A0710A0E3301080E50000A0E1681090E5080011E3FCFFFF0A92
:2001C000E4FFFFEA00FCFFFF0001480001060000051C191030402DE900C0A0E10000A0E375
:2001E000290000EA38E09CE5F4439FE5004094E504001EE12400000A38E09CE52E0852E1AC
:200200000200009A38E09CE52EE8A0E1000000EA02E0A0E10E30A0E1032042E0400053E34B
:200220000000002A0020A0E3040000EA58E09CE5FF400EE200E0A0E1010080E20E40C1E761
:2002400003E0B0E1013043E2F7FFFF1A38E09CE58C439FE5004094E504E0CEE138E08CE504
:200260007CE39FE500E09EE502005EE30300001A40E0A0E368439FE500E084E5020000EAD1
:2002800002E0A0E358439FE500E084E5000052E3D3FFFF1A3040BDE81EFF2FE104E02DE539
:2002A0000030A0E100C0A0E3400052E30100002A0200A0E1000000EA4000A0E300C0A0E139
:2002C0000C2042E0010000EA0100D1E4540083E50C00B0E101C04CE2FAFFFF1A340093E529
:2002E000100080E3340083E51A0000EA400052E30100002A0200A0E1000000EA4000A0E31B
:2003000000C0A0E10C2042E0010000EA0100D1E4540083E50C00B0E101C04CE2FAFFFF1A53
:200320000000A0E1340093E5010010E3FCFFFF0A340093E50100C0E3340083E50000A0E12B
:20034000340093E5010010E3FCFFFF1A340093E5100080E3340083E5000052E3E2FFFF1AFF
:200360000000A0E1340093E5010010E3FCFFFF0A340093E50100C0E3340083E50000A0E1EB
:20038000340093E5010010E3FCFFFF1A0200A0E104E09DE41EFF2FE130402DE90030A0E15D
:2003A00040429FE50E0000EA0350A0E10030D1E5011081E2053023E008C0A0E3050000EA9F
:2003C00003E0A0E1A330A0E101001EE30000000A043023E001C04CE200005CE3F7FFFF1AE5
:2003E000012042E2000052E3EEFFFF1A0308A0E12008A0E13040BDE81EFF2FE1F0402DE9C0
:200400001148A0E30050A0E30070E0E30000A0E1020000EA040094E4007007E0015085E202
:20042000200055E3FAFFFFBA010077E30200001A0000A0E3F040BDE81EFF2FE1A8219FE569
:200440001118A0E30000A0E3D2FFFFEB0060A0E198019FE5BE1FD0E1060051E10100000AE3
:200460000000A0E3F2FFFFEA0100A0E3F0FFFFEAF0402DE984D04DE274619FE574719FE538
:200480000206A0E3400090E56C119FE5010050E10200000A0FE0A0E116FF2FE14C0000EA12
:2004A0000000A0E30216A0E3400081E5080000EA380097E5420000E224119FE5000081E58F
:2004C000000081E2000090E5000050E30000000A000000EAF5FFFFEA0000A0E10120A0E31B
:2004E00004108DE20700A0E139FFFFEB0400DDE5060050E30000000A330000EA0000A0E326
:200500000400CDE50120A0E304108DE20700A0E161FFFFEB0220A0E304108DE20700A0E17C
:200520002BFFFFEBB440DDE1370B54E30000000A250000EA0220A0E304108DE20700A0E1B3
:2005400023FFFFEBB400DDE1030050E30000000A1D0000EA0050A0E3020000EA0500A0E191
:2005600019FF03EB015085E2100055E3FAFFFFBA7C509FE5080000EA8020A0E304108DE2DB
:200580000700A0E112FFFFEB0510A0E104008DE2DAFE03EB804044E2805085E2000054E3B5
:2005A000F4FFFF1A0000A0E30400CDE50120A0E304108DE20700A0E137FFFFEB3C009FE567
:2005C0000010A0E3000301E50000A0E10000A0E1FEFFFFEA0000A0E384D08DE2F040BDE89C
:2005E0001EFF2FE10010200008840000FEDB000000DB1100002010000000FBFF2143341279
:20060000010000A50000A0E11A0000EB03002DE9740000EB0300BDE83C0000EB0F002DE942
:20062000730000EB0F00BDE81CC09FE50FC08CE001001CE30DE08F120FE0A0011CFF2FE1C4
:2006400001C08FE21CFF2FE100F010F83CFEFFFF01402DE90000A0E1930000EB0140BDE8D1
:20066000000000EB0000E0E3A3FEFFEB0400C046C046200000F020F90E40A0E1600000EBEE
:2006800004E0A0E101402DE9750000EB0040B0E10140BDE80010B0E1000084E51EFF2FE150
:2006A00010402DE903002DE96D0000EB0040B0E10300BDE8002094E50D30A0E100E082E051
:2006C00003005EE1002081E50B00008A0E3093E0011A8EE26330A0E1071081E20730C3E316
:2006E0000710C1E3030051E10310A081001084E51040BDE8020041E01EFF2FE10020B0E167
:200700000000B0E30000A0E11040BDE81EFF2FE101C08FE21CFF2FE1F0B505000C0085B05B
:2007200000F0CEF8002001950294C046C046039001A8FFF7D9FC040001A80D00009303C88C
:200740001600C046C046C046C046C046C04600210800C046C046070000F08CF804900021FA
:2007600007600800C046C046411C0498416000210800C046C0460100049881600021080088
:20078000C046C04601000498C16000210800C046C046010004980161C046C046C046C04643
:2007A000C046C046C046C046C046C046C046C046C046C046C046C046C046C046009B05B095
:2007C0002000049C29003200A646F0BC01B0704710B50020C046C046C046C046C046C046F5
:2007E00010BC08BC184700000000E0E30210E0E31EFF2FE110402DE90000A0E11040BDE869
:200800001EFF2FE10E50A0E1200000EB05E0A0E10050B0E10D10A0E10A30A0E10700C0E377
:2008200000D0A0E160D08DE220402DE935FEFFEB2040BDE80060A0E30070A0E30080A0E357
:2008400000B0A0E30710C1E305C0A0E1C009ACE8C009ACE8C009ACE8C009ACE801D0A0E19E
:200860001EFF2FE104009FE51EFF2FE11EFF2FE1141020007847C04604009FE51EFF2FE1AB
:200880001EFF2FE12410200010B410BC7047000000009FE51EFF2FE10410200004009FE523
:2008A0001EFF2FE11EFF2FE10810200000C09FE51CFF2FE1D10710007847C04663FFFFEA3F
:2008C0007847C04610402DE9F3FFFFEB0010A0E3001080E51040BDE81EFF2FE10C091000C2
:2008E000000120001801000094001000240A1000001020000400000094001000280A1000C2
:200900000410200060000000BC00100004E02DE50136A0E12336A0E12020A0E3020000EA40
:2009200004C090E404C083E4012042E2000052E3FAFFFF1AE0C09FE581C00CE001C08CE347
:200940005AC48CE300E0A0E39CC00EE50000A0E100C0A0E398C01CE501001CE3FBFFFF0A38
:2009600004E09DE41EFF2FE110402DE90040A0E3040000EA011684E2021A81E2110884E253
:20098000E1FFFFEB804084E2370B54E3F8FFFFBA1040BDE81EFF2FE110402DE980D04DE237
:2009A0000040A0E3030000EA0000E0E300108DE2040181E7014084E2200054E3F9FFFFBA29
:2009C0001118A0E300008DE2CFFFFFEB80D08DE21040BDE81EFF2FE10F0000E20010A0E3DF
:2009E000981011E50120A0E31220A0E1020811E10300000A24109FE5001481E10020A0E328
:200A00009C1002E50000A0E10010A0E3981011E5010011E3FBFFFF0A1EFF2FE100FF03006A
:200A20000400005A00000000FFFFFFFFFFFFFFFFFFFFFFFFFFFFFFFFFFFFFFFFFFFFFFFF70
:200A4000FFFFFFFFFFFFFFFFFFFFFFFFFFFFFFFFFFFFFFFFFFFFFFFFFFFFFFFFFFFFFFFFB6
:200A6000FFFFFFFFFFFFFFFFFFFFFFFFFFFFFFFFFFFFFFFFFFFFFFFFFFFFFFFFFFFFFFFF96
:200A8000FFFFFFFFFFFFFFFFFFFFFFFFFFFFFFFFFFFFFFFFFFFFFFFFFFFFFFFFFFFFFFFF76
:200AA000FFFFFFFFFFFFFFFFFFFFFFFFFFFFFFFFFFFFFFFFFFFFFFFFFFFFFFFFFFFFFFFF56
:20200000591900EAFEFFFFEAFEFFFFEAFEFFFFEAFEFFFFEAFFFFFFFF00F09FE520FF1FE539
:20202000D4152000FFFFFFFFFFFFFFFFFFFFFFFFFFFFFFFFFFFFFFFFFFFFFFFFFFFFFFFFB3
:20204000000000000000000000000000000000004A2D4C696E6B2041524D20563820636FDB
:202060006D70696C6564204D617920323720323030392031373A33313A323200436F7079CB
:20208000726967687420323030332D32303039205345474745523A207777772E73656767D5
:2020A00065722E636F6D0000000000000000000000000000000000000000000000000000DC
:2020C000FFFFFFFFFFFFFFFFFFFFFFFFFFFFFFFFFFFFFFFFFFFFFFFFFFFFFFFFFFFFFFFF20
:2020E000FFFFFFFFFFFFFFFFFFFFFFFFFFFFFFFFFFFFFFFFFFFFFFFFFFFFFFFFFFFFFFFF00
:2021000070B50C4C0C4E82B02500241D03E008F019F80C350C34B54208D2616820682A682F
:202120008142F4D1002108F019F8F2E702B070BC01BC00479CAB1000CCAB100001C08FE222
:202140001CFF2FE1044C054D054E064FAE462047002809D0BE463047B98010005121100068
:202160000121100069211000044C054D0020AE462047044C044DAE4620470000B1A0100019
:202180007321100011A1100075A1100000B581B068461D210170052105F02CF801B000BDC3
:2021A00000B582B0694600220A604A600870020A4A70020C8A70000EC8702121684605F0E2
:2021C0001FF802B000BD000010B583B0040001A80021016041606846052101700221417098
:2021E0000521401C05F006F80521684605F008F8FFF7CCFF210312480843FFF7D1FF012030
:2022000004F07AFF68460C2181700521801C04F0F1FF222101A804F0F3FF040004F082FF94
:202220002000203004F080FF0006000EC007F0D504F078FF200004F08DFF03B010BDC0468A
:20224000150E00EE30B583B005000C0001A800210160416068460521017002214170052139
:20226000401C04F0C7FF0521684604F0C9FFFFF78DFF290314480843FFF792FF684600210D
:2022800081700521801C04F0B5FF01A80470210A4170210C8170210EC170222104F0B0FF86
:2022A000012004F029FF222101A804F0A9FF040004F038FF2034200004F036FF0006000E79
:2022C000C007F0D503B030BD150E10EE10B582B00400FFF75BFF2000FFF762FF012004F0DA
:2022E0000BFF6846002101604160FFF74FFF2121684604F085FF040004F014FF20342000D8
:2023000004F012FF0006000EC007F0D502B010BDFAB585B00500160003A8002101604160CC
:20232000059C724802681F218A431321114301600020FFF787FF6E48FFF7C8FF290000208A
:20234000FFF780FFE80710D5002C0ED06448FFF7BDFF0120FFF738FF0106090E0698017051
:202360000698401C06906D1C641E700079D4022005420DD0022C0BD35A48FFF7A7FF012054
:20238000FFF722FF0104090C06A807F041FEA41E300052D4042C50D3A50805266846C67001
:2023A00002210171052101A804F024FF310000A8C01C04F025FF68460C214171310001A86E
:2023C000401C04F017FFFFF7E1FE4748FFF7E8FE68468670022141703100401C04F00AFF55
:2023E000310000A8801C04F00BFF68460C210170310004F0FFFE002D1DD02E00012004F09F
:202400007BFE222103A804F0FBFE070004F08AFE3800203004F088FE0006000EC007F0D543
:2024200004F080FE380004F095FE010006A807F0F7FD761EE2D1A800241A022C11D3650825
:202440000DD02E002748FFF741FF0120FFF7BCFE0104090C06A807F0DBFD761EF2D16800A5
:20246000241A002C0FD01E48FFF730FF0120FFF7ABFE0106090E069801700698401C06900B
:20248000641EF0D1002402A800210160684601210170022141700521401C04F0ABFE05214F
:2024A000684604F0ADFE68460C2181700521801C04F0A0FE202102A804F0A2FE050004F037
:2024C00031FE280004F046FE410601D4000602D50020C04301E00598001B07B0F0BDC0464E
:2024E0000110D0E4B210D0E0015EB0EC9C00200000F02FE1F2B584B0060017001D0002A82F
:20250000002101604160049C6A4802681F218A431321114301600020FFF794FE6648FFF79A
:20252000D5FE31000020FFF78DFEF0070BD5002C09D029786D1C0120FFF784FE5A48FFF7BF
:20254000C5FE761C641E780075D4022006420FD0022C0DD3C1480178280007F077FD010076
:202560000120FFF76FFE5148FFF7B0FEAD1CA41E38004AD4042C48D3A00801906846052161
:202580008170022141700521401C04F033FE052100A8801C04F034FEFFF7F8FD4448FFF7D2
:2025A000FFFD684600210170052104F023FE0198002827D00600A9480178280007F06AFDF6
:2025C00001006846017202A80A0A42700A0C8270090EC170222104F013FE012004F08CFD33
:2025E000222102A804F00CFE070004F09BFD2037380004F099FD0006000EC007F0D52D1D5A
:20260000761ED8D101988000241A022C13D366080FD0370091480178280007F017FD010008
:202620000120FFF70FFE2148FFF750FEAD1C7F1EF0D17000241A002C0AD029786D1C0120A3
:20264000FFF700FE1848FFF741FE641EF5D1002401A8002101606846012101700221417045
:202660000521401C04F0C6FD0521684604F0C8FD68460C2181700521801C04F0BBFD202119
:2026800001A804F0BDFD050004F04CFD280004F061FD410601D4000602D50020C04301E02A
:2026A0000498001B05B0F0BD0110C0E4B210C0E0015EA0EC9C00200000F02FE1F0B584B06A
:2026C0000024E443042102A804F04EFF0421684604F04AFF009803900002000A00900500C3
:2026E0008020C000854201D2019500E00190019804F050FE06001BD0002D17D00198854299
:2027000001D22F0000E007003300039A39000298FFF7FEFD04000DD40298001902902D1BCA
:202720002100300004F0CAFEBC42E5D00098441B002D02D0280004F0CBFE002E02D03000CE
:2027400004F04CFE200004B0F0BD0000F0B584B00025ED43042102A804F006FF04216846F1
:2027600004F002FF009803900002000A009004008020C000844201D2019400E00190019801
:2027800004F008FE06000FD1002C02D0200004F0F7FE002E02D0300004F020FE280004B034
:2027A000F0BD029840190290002C17D00198844201D2270000E00700E41B3900300004F038
:2027C000D3FE3300039A39000298FFF793FE0500DAD4BD42E5D00025ED43D5E7009DDAE728
:2027E000F1B592B00221684604F0BEFE6846018802A804F0B9FE02A807F040FC1649086040
:2028000002A80179019145798679C7791349007A08708020C00004F03DFD0022310038009E
:2028200004F064FD01990906090E280004F068FD12A80078642802D0652803D005E0FFF737
:202840003DFF01E0FFF782FF040004F03BFD200004F070FE13B0F0BD9C0020007A0E20005E
:20286000F0B5824C2068C01DC5087E4E30687E4F2A00396849104118401907F015FC68003C
:202880003168091831603968081A386000202060F0BD00007348006870470000F0B588B08E
:2028A00004000D001600714800680790012E61DB092E02DB0820009000E000962F006846AF
:2028C00004736A4800684107490F0191C0086549096808180290644800684010029908187D
:2028E000059008200199411A009807F085FB019900291CD0029A511C069113789C463F0616
:202900003F0E019B3900994063461943117005990491491C049A04B41278944601AA137BAB
:20292000029A93406246134304BC13700AE002990F700299491C069105996A46127B0A70F7
:202940000599491C009A824208D0069A3F063F0E074117706A46127B02410A70434843492C
:202960000968009A891801600098361A240A2D0A012E9DDA079808B0F0BD000010B504008A
:20298000082C07DB0822FF210020FFF787FF083C082CF7DA012C06DB012201210020FFF789
:2029A0007DFF641EF6E710BD224800210160704700B520480168002901D0491E016000BDC7
:2029C000F0B5070003F0B6FE00282BD1194C052F01D22060F0BD1E4D134E2068002809D092
:2029E00064202060306800281CD003F0A7FE01202870F0BD802F15D304F0B2F801000129C9
:202A000010DB0A4807F0C4FB08000949884205D330600121297003F091FE01E00020306069
:202A200064202060F0BDC046A800200000A3E11141420F00AC00200010B5054C207800284E
:202A400004D0002003F07AFE0020207010BD00007B0E2000034A106003480160034800211C
:202A600001607047A0002000A40020006C0420000023C3604261016089184160891881601C
:202A800070470000F0B504000F00E5687E686069C0007119884201D202F0D2FE3F68330048
:202AA0003A00E1682068FEF0F5FD3300F01DC0083A18E168A068FEF0EDFDE0688019E06087
:202AC0002800F0BD00B5C168C91DCB080021C16042688168006803F0C1FE00BD30B50400F5
:202AE000E068C01DC5080020E060E900A06803F087FC2B006268A168206803F0AFFE0028CF
:202B000001D103F0F7FD30BDF0B50400164D2E686436D3492000FFF7B5FF8D490988471827
:202B20002000FFF7DBFF00281CD1F80861680A1810787B075B0F06D0D84001005078082250
:202B4000D21A9040084319210140092901D10020F0BDC00601D50320F0BD2868301A0128B3
:202B6000D7DA0220F0BD00005C03200010B59EB0040003F0BFFD002820D12069C10862685B
:202B800051180A784007400F06D0C24013004A780821081A82401A4319201040092801D111
:202BA00000200BE0D00601D5032007E0202206A96846FFF75DFF6846FFF7A6FF1EB010BD7F
:202BC000F5B583B00C00002001900090009801210140182041435D4845180E2C01D22600DF
:202BE00000E00E2604980068B0426BD00098C00701D5002000E03000049908609549280020
:202C0000FFF740FF07000120B040401E4000029045494018FEF0FCFC444909887B185A0759
:202C2000520F0100D8082B681818FEF00DFD8A492800FFF727FF3E493E4A128880180860D7
:202C4000022E06D3771E84492800FFF71BFF7F1EF9D182492800FFF715FF0700029836494D
:202C60004018FEF0D5FC01003448008838184207520FC0082B681818FEF0E6FC78492800FA
:202C8000FFF700FF3249098840182861E968C91D07208143A86803F0B3FB0E2E15D1E8680D
:202CA000C01DC7083A0029682A48006807F0FCF93A00A9682248006807F0F6F921482969D9
:202CC000016002E020480068E86033001848026803992800FEF0D8F803900198002807D0EF
:202CE000FFF744FF002803D01B490E340C6018E01548E96801602800FFF7E4FE002801D08E
:202D00001549F3E7A41B0098401C00900195002C00D05BE72800FFF729FF002801D00E49CE
:202D20000E6005B0F0BDC046000090E8C800200098012000C60020000000A0E8CA0020004C
:202D400078012000800120009C01200058012000CC002000700120008801200010B5394A95
:202D60001488394B18605C605388E41DE410640004193648046043609088DB1DDB105B00D3
:202D8000E418334B1C605860D388C01DC010400024183048046043601089DB1DDB105B00AB
:202DA000E4182D4B1C6058605389C01DC010400024182A48046043609089DB1DDB105B0096
:202DC000E418274B1C605860D389C01DC01040002418244804604360908CDB1DDB105B00FF
:202DE000E418C34B1C605860D38CC01DC01040002418484804604360108DDB1DDB105B009B
:202E0000E418454B1C605860538DC01DC01040002018424C20606360DB1DDB105B00C31803
:202E20001148124C002909D0518E23606160C91DC910490059180160918E00E0616041607B
:202E400010BD0000B0002000E80020000001200008012000100120001801200020012000D8
:202E6000F0002000F80020005001200048012000F0B581B004001500224E002B37D1254950
:202E8000FFF700FE07000120A84040001E494018FEF0BEFB01001D48008838184207520FA0
:202EA000C00823681818FEF0CFFB1B4F39002000FFF7E8FD1649098840180090022D06D359
:202EC0006D1E39002000FFF7DDFD6D1EF9D113492000FFF7D7FDE168C91D07208143A06881
:202EE00003F08EFAE06830600098206101E03068E0602000FFF7E6FD002801D103F0FAFBD2
:202F000001B0F0BDA0012000FEFF7FE8E0002000DC00200030012000380120004001200027
:202F2000F1B5130002692E480078002834D0002B50D0FF24284DD008009E76683618500777
:202F4000400FB707FF0EC0190327BE433768002808D0C740BC4676682027381A86406746C1
:202F60003E4337001D48006812183E0A2740E85D0706FF203040285C00043843360A2700A8
:202F80003740EF5D3F020743300A285C38430860091D5B1E1ED0CEE7002B1BD0D008009C76
:202FA000646820185407640F8507ED0E64190325A8430568002C06D0E5402E004568202079
:202FC000001B854035430548006812180D60091D5B1EE3D101B0F0BD78AD10003C0120000A
:202FE000D0002000F1B591B00C0000250D2C01D2260000E00D263D4F002D04D00D2E02D1E9
:203000000120009031E00020009039493800FFF739FD0120B040800032494018FEF0F8FA14
:203020000100314800884207520FC0083B681818FEF00AFB2F493800FFF724FD2E49098887
:2030400040183861F968C91D07208143B86803F0D7F9F86801903800FFF734FD00283ED1E3
:203060003800FFF783FD002839D1009B721C03A938001830FFF7FCFE002830D11A2C12D3D7
:203080000198F8603800FFF71DFD002827D1721C03A938001830FFF743FF3800FFF766FD54
:2030A00000281CD105E0721C03A918373800FFF737FF0398C006C00E1F2801D004200EE0D0
:2030C000B7003A0003A9091D119806F0EDFF1198C0191190A41B6D1C002C87D1002012B0D1
:2030E000F0BDC046FCFFAFE8DE0020005801200028012000F0002000CC002000FCB5D24C00
:20310000A54404000D00002004900890059080267600320009A9CD48FFF7AAFC3200C02011
:20312000800009A90918CA48FFF7A2FC07952800FFF746FC052D0CD2C6494868002808D0CB
:20314000C248FFF79FFCC148FFF7C8FC070000D052E1C149BD48FFF795FCC0480190007C5C
:20316000002803D02000FEF053FA00E0200001990B885A07520F0100D808B44B1B68181877
:20318000FEF062FAB148FFF7A9FC070000D033E1E0072BD500200290012102A8B04A6A4459
:2031A0001268126806F0E8FE6D1E0198007C002803D00298FEF02CFA0290AC49A348FFF78E
:2031C00061FC0199498840184207520F0299C0089E4B1B681818FEF037FA9C48FFF794FC9D
:2031E000070002D00120049006E1641C02210C4235D0022D33D3002000906846984A6A4441
:203200001268126806F0B8FEAD1E0198407C002805D000980004000C06F0B0FE009001987C
:20322000007C002803D00098FEF0F2F900908E498648FFF727FC0199898840184207520FAB
:203240000099C008814B1B681818FEF0FDF97F48FFF75AFC070001D00220C4E7A41C042D01
:2032600052D304F085F80200382106F089FF101A069004F08FF80590A80880000699884276
:2032800001D2039000E0039103990598744A6A441268526806F070FE002000907048684403
:2032A0000068806806F030FF0399091A03229143009A8E1A002806D0382EEFD330003821F0
:2032C00006F05EFF361A002F10D108AAB108009880088000059B1818FFF772FC0700A41938
:2032E000002F03D05F4800688000241A00988019009003998842D1D16D1A042DBCD2002FC1
:2033000002D00420049077E002210D4232D0002000906846524A6A441268126806F02CFE9C
:20332000AD1E0198407C002805D000980004000C06F024FE00900198007C002803D0009878
:20334000FEF066F9009048494048FFF79BFB0199898840184207520F0099C0083B4B1B68D4
:203360001818FEF071F93948FFF7CEFB070000D072E7A41C002D28D00020009001216846F0
:20338000374A6A441268126806F0F6FD6D1E0198007C002803D00098FEF03AF900903349C1
:2033A0002A48FFF76FFB0199498840184207520F0099C008254B1B681818FEF045F92348B3
:2033C000FFF7A2FB070000D00CE729491F48FFF759FB1E48FFF782FB07000DD107980528E3
:2033E0000AD224494868002806D01848FFF74AFB1648FFF773FB0700002D09D0012102A8A0
:20340000174A6A441268126806F0B6FD6D1EF5D1C520C00068440068390007800AD0C52077
:20342000C000684400684460C520C0006844006804994180059803F0D1FFFFF7FDFA380078
:203440000D498D44F0BDC046DCF9FFFF580120007001200048012000E8002000C000200064
:2034600024060000880120000801200000012000F8002000500120002C06000070B585B01A
:203480000121684604F070F86846007801281ED01F4C002801D1242102E0022803D13221E6
:2034A000200004F061F81B4D280003F0A9FFE08B03F070FF06002E6001D102F0C1F9E18B29
:2034C000300004F051F800213000FFF747FC042101A804F049F8042102A804F045F803AB44
:2034E0000A4A02990198FFF709FE03AC20880006000E04F00FF82088002805D0049804F0AC
:2035000019F8608804F016F805B070BDECAC1000B000200094012000FFB5C34CA5440020D5
:203520000390009008900690C04C80256D002A000AA92000FFF79CFA2A00C02080000AA956
:20354000091820001830FFF793FAB948684400680490B74868440068FFF732FA03F008FF87
:20356000079003F017FF0990B2492000FFF78AFAB1480078002806D0C520C0006844006855
:20358000FEF046F803E0C520C00068440068AB490B885A07520F0100D80823681818FEF090
:2035A00053F82000FFF79AFA0090099D04980799884201D2059000E00591059E0098002899
:2035C00000D043E1C520C00068440068C0073ED501200390761EC7492000FFF753FAC6489B
:2035E000FEF016F8C5490B885A07520F0100D80823681818FEF028F82000FFF785FA002805
:2036000016D10023022201A92000FFF731FC00280ED1022201A92000FFF782FC0198C006C7
:20362000C00E1F2801D0042002E00298287000200090002800D009E16D1CC520C000684400
:203640000068401C02B47A496944086002BCC620C00068440068400000D5B6E0C520C00050
:20366000684400680221084242D0022E40D30391B61EA0492000FFF705FAA148FDF0C8FF71
:203680009E490B885A07520F0100D80823681818FDF0DAFF2000FFF737FA002819D1002310
:2036A000022201A92000FFF7E3FB002811D1022201A92000FFF734FC0198C006C00E1F28B6
:2036C00001D0042005E0029828700298000A687000200090002800D0B8E0AD1CC520C000B4
:2036E00068440068801C02B451496944086002BCC620C0006844006800002CD4042E2AD30E
:20370000B70804200390B800361A39002800FFF769FC0090002800D098E0B8002D18C5208D
:20372000C00068440068B90040180FE0029828700298000A687000200090002800D085E0FA
:20374000AD1CC520C00068440068801C02B438496944086002BC022E37D302200390B61E7E
:2037600064492000FFF78EF96548FDF051FF63490B885A07520F0100D80823681818FDF08B
:2037800063FF2000FFF7C0F90028D5D10023022201A92000FFF76CFB0028CDD1022201A928
:2037A0002000FFF7BDFB0198C006C00E1F28BDD00420C1E76D1CC520C00068440068401CD0
:2037C00002B41B496944086002BC002E3ED001200390761E47492000FFF754F94648FDF00A
:2037E00017FF0100454800884207520FC00823681818FDF029FF2000FFF786F9002822D1AB
:203800000023022201A92000FFF732FB00281AD1022201A92000FFF783FB0198C006C00ED2
:203820001F280DD004200EE0D8F9FFFF580120002C060000E8002000D0002000C000200000
:2038400002982870002000900028B3D00698002823D1012168462B4A6A441268126806F044
:203860008BFB00980890002817D0284868440068412815D30421C520C0006844214A6A441F
:203880001268126806F078FB042103A81D4A6A441268126806F070FB22E00898002804D0F3
:2038A0001A4868440068412807D205990998164A6A441268126806F05FFB04980599401A2B
:2038C00004900698401C06900498002800D06CE60098002804D00D48684400684128C9D3DC
:2038E000099803F07BFDFFF7A7F80898C721C9008D44F0BD280120000120D0E4DE0020003C
:20390000B220D0E04C060000340600002C060000F0B581B004000D006C4886784078401EB8
:20392000871B032200210120FEF7B8FF002F04D03A0000210020FEF7B1FF4C480068009023
:2039400008E000203A0021780006000EFEF7A6FF641CED1B012D0CDB082D01DA2F0000E022
:203960000827002EEDD1092DEBDA0120691E8840E8E7002E06D0320000210120761EB040F6
:20398000FEF78CFF012200210120FEF787FF009801B0F0BDF1B54D4C6078012822D1012578
:2039A0006846007804214E1B0121B140491E014001222A41914212D1042200210320FEF7F5
:2039C0006DFF2A006846017831410906090E01206D1EA8400006000EFEF760FF3FE06D1CEE
:2039E000052DDFDB21480068002803D101220021FEF754FF04276D46E6782078001F841BF0
:203A0000042200210320FEF749FF002C05D02000FEF7B4FF01E0082F01DA3C0000E00824FB
:203A2000002E05D1092F03DA0120791E884000E00020220029780006000EFEF72FFF6D1C6A
:203A40003F1B012FE7DA002E09D0022E02DB701EFEF794FF012201210800FEF71FFF01226E
:203A600000210120FEF71AFF01B0F0BD6C04200070B581B00500154E3079002801D005247F
:203A800000E004240220FFF785FF0120611E8840210000957278012A12D14A1E10D08B1A7F
:203AA0000400DC40009B012595406D1E1D40AC4204D1891A1800D040009001E0521EEED13A
:203AC0006846FFF725FF01B070BD00008C01200010B582B004005F480078002810D1200050
:203AE000FDF096FD40006946087002124A7002148A700016C87001202040087121210EE089
:203B00002000FDF085FD6946C2000A7042094A70420B8A70420DCA70400F0871232168469C
:203B2000FFF7F6FE0400012200210020FEF7B6FE200002B010BD000070B582B00500504EF1
:203B40004448007800281DD102243000FDF060FD400001210143684601700A1242700A14FA
:203B600082700916C170002101712121FFF7D0FE012200210020FEF791FE2800FFF7A8FFBD
:203B800005001DE004242800FFF7A2FF05003000FDF03EFD6A46C300042119431170410920
:203BA0005170410B9170410DD170400F107123216846FFF7ADFE012200210800FEF76EFE58
:203BC0000420FFF7E7FE04E0012200210020FEF765FE2000441E0028F6D1280002B070BDCE
:203BE00010B5012404E0012200210020FEF756FE2000441E0028F6D110BD000010B583B014
:203C000014490978002902D1FFF762FF1FE06C462070010A6170010CA170000EE07018487A
:203C2000FDF0F6FCC100217141096171410BA171410DE171400F207243216846FFF768FEE9
:203C40000400012200210020FEF728FE200003B010BD00009001200010B50400012C0DDBB2
:203C60000748FFF735FF641E04E0012200210020FEF714FE2000441E0028F6D110BD0000BC
:203C80000000A0E110B582B06A4611606946202202430A7126216846FFF73AFE012404E0AE
:203CA000012200210020FEF7F9FD2000441E0028F6D102B010BD000000B50120FFF7D8FE23
:203CC0000C20FFF767FE00BDF0B584B00400DC4F787803903879002802D10125009502E0CC
:203CE000002503200090012200210020FEF7D6FDFFF7E2FFA748FFF7EBFE3879002802D070
:203D00000220FFF7A9FFA448FFF7E2FEA348FFF7DFFE3879002802D00420FFF79DFFA0481A
:203D2000FFF7D6FE0220FFF797FF0020FFF766FF06003879002801D1FFF752FF701920826D
:203D40000F20FFF727FE9C4E30682080FEF788FDFFF7B2FF9348FFF7BBFE0220FFF77CFFB9
:203D60000020FFF74BFF40196082FFF739FF9348FFF7AEFE8C48FFF7DFFE30686080FEF7E9
:203D80006FFDFFF799FF8748FFF7A2FE0220FFF763FF0020FFF732FF4019A082FFF720FF73
:203DA0008648FFF795FE8148FFF7C6FE3068A080FEF756FDFFF780FF0020FFF789FE00997E
:203DC000401820837A4803990129397912D0002904D1FFF77DFEFFF703FF02E00220FFF76B
:203DE0003BFF3068E080FEF73BFD0020FFF706FF401918E0002904D1FFF76AFEFFF7F0FEB8
:203E000001E0FFF765FE3068E080FEF729FD3879002803D1FFF7F2FE401904E00020FFF76F
:203E200057FE00994018E08230682081FEF718FD3879002804D1FFF7D3FEFFF7D1FE02E07B
:203E40000520FFF709FF0020FFF776FE00994018608330686081FEF703FD0122002100200F
:203E6000FEF71CFD0220FFF703FE0C20FFF792FD01A8002101604160684601210171062135
:203E800001A8FFF745FD684600210171052101A8FFF73EFDA0833068A081FEF7E1FC0F2023
:203EA000FFF778FD3068E081FEF7DAFCFFF704FF4248FFF70DFE0020FFF73EFE009940180C
:203EC000E0853068A084FEF7CBFCFFF7F5FE3948FFF7FEFD3879002802D00220FFF7BCFE2D
:203EE0000020FFF7F5FD0099401820860220FFF7B3FE3068E084FEF7B3FC3879002802D10E
:203F00000020C04300E02D48FFF7E2FD4019A08530682085FEF7A4FC0F20FFF73BFD30680F
:203F20006085FEF79DFC0220FFF7A2FD0C20FFF731FD0021C9430B20FFF7A4FE00210920CD
:203F4000FFF7A0FE00210820FFF79CFEF7210D20FFF798FE802149000C20FFF793FE0F2057
:203F6000FFF718FD894C30686086FEF779FC0220FFF77EFD0C20FFF70DFD00210C20FFF777
:203F800081FE0F20FFF706FD3068A086FEF768FC04B0F0BD00000FE1DF0080E300F02FE1D0
:203FA00001009EE8020090E80110C0E4B210C0E0FFFFFFEA00100FE16C0420000000A0E1F1
:203FC000F0B504000D001D4E1D4FB078A84206D108222100380006F0A1F800282DD008220A
:203FE0002100380006F060F8694C200003F008FA8020000103F0CEF9206080210901FEF7D5
:2040000029FD00203979002901D1012100E000213170002D00D03078B070787970705B48B0
:20402000FFF752FEFEF736FC2268811A100003F0DDF901212068FEF791FEF0BDD00020004A
:204040008C01200000B508220021024806F086F800BD00008C01200000B5FFF7F3FFFFF7F8
:204060000DFA00BD70B583B0FFF7ECFF012101A803F07AFA6846007901281ED0434C00281C
:2040800001D1242102E0022803D13221200003F06BFA3F4D280003F0B3F9E08B03F07AF93A
:2040A00006002E6001D101F0CBFBE18B300003F05BFA00213000FEF751FE042102A803F0A8
:2040C00053FA0421684603F04FFA009A1002000A0090304B08B401000398FFF71DFA04B0AA
:2040E00070BD000000B582B00821684603F03CFA00216846FFF764FFFFF7C0F902B000BD66
:2041000070B585B0082103A803F02EFA002103A8FFF756FF012101A803F026FA684600793A
:2041200001281ED0194C002801D1242102E0022803D13221200003F017FA154D280003F0F0
:204140005FF9E08B03F026F906002E6001D101F077FBE18B300003F007FA00213000FEF7EB
:20416000FDFD042102A803F0FFF90421684603F0FBF9009A1002000A0090064B08B401007D
:204180000398FFF7C9F906B070BD0000B000200094012000F8AC1000F0B5FFB0EFB0082293
:2041A000AD490CA805F080FF0821AB4803F0DCF90221684603F0D8F9022100A8801C03F00E
:2041C000D3F9022102A803F0CFF9022102A8801C03F0CAF968460488802189000EA8FEF75D
:2041E00039FC924D92480078E872012200210020FEF754FB0220FFF73BFC0C20FFF7CAFB21
:20420000934E30682880FEF72BFB04A8002101604160684604210174062104A8FFF778FB0F
:20422000002768460774062104A8FFF771FBE88130686880FEF714FB06A8076047606846A2
:2042400005210176062106A8FFF762FB68460776202106A8FFF75CFB28823068A880FEF7D3
:20426000FFFA0F20FFF796FB3068E880FEF7F8FA298870480EAA02606F4801606888C91D37
:20428000C910490052186D490A606D490860A988C01DC010400012186A4F3A6079606A482E
:2042A000C91DC9104900511801606848E9880160684E40228EA93000FEF7DAFB40228EA9C8
:2042C000C03130001830FEF7D3FB68460088800003F060F80190002832D056493000FEF732
:2042E000D1FB3000FEF7FAFB019803905B480068694609894018089050493000FEF7C2FBF5
:20430000F168C91D07208143B06802F079F8F0680990390030001830FEF7B4FB716AC91DF1
:2043200007208143306A02F06BF8706A0A90200072D145493000FEF7A5FB3000FEF7CEFB8B
:2043400068460088041B200003F0F4F8A100019803F0B4F80198002801D003F03FF808224A
:204360000CA93D4805F0A0FE7FB06FB0F0BD0B983A490968401AE3D4089838490968401AE1
:20438000DED40998F0603000FEF79CFB002801D102F0B0F90028D3D1E989C8087268101819
:2043A0004907490F03220240D2008918B8430268002906D0CA40130042682020401A8240F4
:2043C0001A439007D3D50A98706230001830FEF779FB002801D102F08DF90028B0D1298A1E
:2043E000C808F26910184907490F0740FA008918032290430268002906D0CA4013004268B8
:204400002020401A82401A43039802600398001D0390641E2404240C20008AD00F48006888
:204420006946498840180B900327A5E7A401200091012000B8012000BC012000C001200045
:20444000C4012000C8012000D0012000D40120006C042000580120008C0120005C03200073
:2044600000B503480068000EFF2800D1002000BDD8012000024800784007400F7047C046E3
:20448000DD01200072480168C90A4068400508437047000000B530236D4A01494E484DE06D
:2044A00034AC100030B504002E23694A004907E03CAC100030B504002E23654A0749C046B8
:2044C000644800F08DFEFFF7D5FF0500012D02D1FFF7D8FF2060280030BDC04644AC10007D
:2044E00030B504002E235A4A0049E9E75CAC100003B569464203BB2313430B60010C4140D4
:204500000A0A4A40110951408A084A406946C00C130052085A40012313405A0302438A8091
:2045200030234B4A2C4800F05BFEFFF7A3FF0CBD00B50823464A03490348C04600F050FE2A
:2045400000BDC0467AAE100078AE1000F3B500248210424001236D468608012737407E00C8
:204560008007C00E30431600521072401E0016407201024381201043A8704801E8706846C2
:20458000CA084260080C4840010A41400809484081084140E8790A00490851400B405901EA
:2045A0000143E97103E02000641C642810D03023274AA91C084800F013FEFFF75BFF06003E
:2045C000012E01D10020FCBDFFF764FF022EEAD00020C043FCBD00002CAC100010B58BB0FA
:2045E00084235B0001AA1649164800F0F9FD2E23174A1549174800F0F3FDFFF73BFF0128C3
:2046000002D1FFF73FFF00906846FFF769FF0024E4430098B221084208D0FFF73BFF684641
:20462000FFF75EFF0098A021084206D1074900910120FFF78BFF002800D020000BB010BD8B
:2046400064AC100088AC100054AC100001000050DC01200024AC100070B504000D00FFF78C
:2046600019FF00210220FFF771FF0600064929430420FFF76BFF0500354321000520FFF77B
:2046800065FF284370BDC04610000023F0B50C000025ED430221FFF7DFFF002819D10026B0
:2046A00003E03000761C642813D02000FFF702FF0700012F09D12000FFF7F4FEFFF7EAFED8
:2046C0002000FFF7EFFE0020F0BDFFF7E3FE022FE7D02800F0BD000010B50C000221FFF78C
:2046E000BBFF002801D0002006E021000720FFF72DFF002802D00120C04310BDFFF718FF9F
:20470000002010BDFAB582B0040017005910FFF7A3FF002802D00020C04375E00190002587
:2047200007E0FFF7B7FE022EF5D128006D1C6428F1D06846FFF7BEFE0600012EF1D1032574
:204740000226019800282CD00398012804D002280CD0042817D022E0009821002940C900D6
:20476000C8400090009838707F1C18E0009802222240D100C8400090009838700098000A65
:204780007870BF1C0BE0009838700098000A78700098000CB8700098000EF8703F1D0398D0
:2047A00024180198401C019002998842B7D36846FFF778FEFFF76EFE6846FFF773FE03981C
:2047C000012804D0022808D0042810D01BE000982540E900C840387015E000982640F10059
:2047E000C8400090009838700098000A0AE0009838700098000A7870BF1C0098000C387064
:204800000098000E7870019804B0F0BDFAB582B0040015000020019059102000FFF71CFFCB
:20482000002802D00020C0433DE0029EA8070AD10398042807D10120019002E00198002820
:2048400001D0286817E02878039902290DDB01006878000208430399032906DB0200A878B8
:204860000104E8780006084310430422039BD21A2240D10088400090002707E00228D1D11A
:2048800038007F1C6428CDD0FFF704FE0098FFF72FFE0128F2D103982D182418761ECDD12F
:2048A000FFF746FE029804B0F0BD0000FCB505000E00002407E03800019988402D1800997C
:2048C00008180090F61B002E1BD0EF43FFF7C8FD032802D13F053F0D01E0BF05BF0D019879
:2048E000C7407F1CBE4200D2370001238340009A39002800FFF706FF002803D42418B842FB
:20490000D9D02000FCBD0000F2B5060017001D000C00C0070FD5002C0DD000232A00012105
:204920003000FFF7C3FF002800D5F8BD241A012846D16D1C761C780037D4B0070FD5022CF8
:204940000DD301232A0001213000FFF7AFFF0028EBD44100641A012832D1AD1CB61C38008E
:2049600011D4042C0FD3A70802232A0039003000FFF79CFF0028D8D48100641AB8421FD18B
:20498000B8002D183618022C0FD3670801232A0039003000FFF78AFF0028C6D44100641A96
:2049A000B8420DD178002D183618002C08D000232A0021003000FFF779FF0028B5D4241A15
:2049C0008AE00000FCB505000E00002407E03800019988402D18009908180090F61B002E37
:2049E0001BD0EF43FFF73CFD032802D13F053F0D01E0BF05BF0D0198C7407F1CBE4200D25F
:204A0000370001238340009A39002800FFF7FEFE002803D42418B842D9D02000FCBD0000D4
:204A2000F2B5060017001D000C00C0070FD5002C0DD000232A0001213000FFF7C3FF002856
:204A400000D5F8BD241A012846D16D1C761C780037D4B0070FD5022C0DD301232A00012197
:204A60003000FFF7AFFF0028EBD44100641A012832D1AD1CB61C380011D4042C0FD3A70817
:204A800002232A0039003000FFF79CFF0028D8D48100641AB8421FD1B8002D183618022C97
:204AA0000FD3670801232A0039003000FFF78AFF0028C6D44100641AB8420DD178002D1859
:204AC0003618002C08D000232A0021003000FFF779FF0028B5D4241A0098001BF8BD000021
:204AE000F3B515000221B448FFF7B6FD040010210220FFF72BFD204304000098017805201F
:204B0000FFF724FD06002643002403E02000641C64281CD02E23154A1349154800F060FB3C
:204B2000FFF7A8FC0700012F0DD1FFF7ABFC019908600198FFF7B6FCFFF7ACFC0198FFF7B9
:204B4000B1FC002005E0FFF7A5FC022FDED00020C04330430099491C00910199091D0191B6
:204B60006D1EC9D1FCBDC0464CAC1000DC01200024AC1000F0B504000D00160002218E48A7
:204B8000FFF76AFD070010210220FFF7DFFC010039430F0029680620FFF7D8FC0100394303
:204BA0000F0020788021490201430520FFF7CEFC38430700641C2D1D761EEBD1FFF7B8FCF3
:204BC0003800F0BD11B57C4C69462000FFF75EFD002810D10098000307D5AC492000FFF7B7
:204BE0007BFD69462000FFF751FD0098800301D5012018BD002018BD00B5A4496E48FFF700
:204C00006BFD002801D1FFF7DDFF00BD10B56A4C002805D005492000FFF75EFD044900E03F
:204C200004492000FFF758FD002010BD0B005FA009005FA001005FA030B50024E4435E4DE2
:204C40000A492800FFF748FD002805D108492800FFF742FD002801D0200030BDFFF7B2FF45
:204C600004008A492800FFF737FDF5E70F005FA00D005FA0F1B501218748FFF72DFD4F4CC3
:204C8000FFF7EEFB032801D14D4900E04D492000FFF722FD7B4C2568FA358026B604464F7F
:204CA00069463800FFF7F2FC0098304002D02568FA3506E02068281AF2D585E02068281AED
:204CC000FBD469463800FFF7E1FC00983040F5D100217148FFF700FD6C49380078E000006B
:204CE000F1B500260024344D02E0FFF777FC012666492800FFF7F0FC01216748FFF7ECFC69
:204D0000FFF7C8FB2D48310001D02D4900E02D49FFF7E2FC69462800FFF7B8FC0099254A3A
:204D20000A4001D1002802D5002EDED04CE055480768FA3706E00068381AF7D469462800D1
:204D4000FFF7A4FC009880014E48F4D50768FA374C480068381AE9D469462800FFF796FC3B
:204D600000988001F4D449492800FFF7B5FC002C07D002214648FFF7AFFCB1214548FFF747
:204D8000ABFC00214448FFF7A7FC002C0FD1052002F0A4FF69462800FFF778FC0098000384
:204DA00001D50124A4E7FFF70DFF0028F9D0374928000DE00000F0FCF0ED00E00CED00E063
:204DC0000100FA050400FA050020C043F8BD0000FFF782FCFFF7F6FEF8BD0000F3B581B00C
:204DE0000026284C284D00E0012628492800FFF773FC01212848FFF76FFCFFF74BFB01204F
:204E000002F06CFF01F064FA019802F067FF01F063FA0298002800D1642002F05FFF2068B8
:204E200017494718FFF7CEFE012802D02068381AF8D516492800FFF74FFC002E07D002215F
:204E40001348FFF749FCB1211248FFF745FC00211148FFF741FC002E0DD1052002F03EFF4C
:204E600069462800FFF712FC00980003BCD4FFF7A9FE0028B8D002990198FFF7FBFEFEBD01
:204E8000DC0500005C032000F0ED00E003005FA00000044004000440FCED00E030B50300B6
:204EA0000C0015000020C043002B04D0012B0DD0022B10D030BD29002000FFF711FF012834
:204EC0000DD029002000FFF789FF30BD29002000FFF7D0FE30BD29002000FFF77FFF30BD9D
:204EE000FFB50024E443042101A802F03DFB0421684602F039FB009803900002000A0090FB
:204F0000050002F035FA06000098B04200D20600300002F03FFA07001BD0002D17D0B542AB
:204F200001D2029500E002963B00039A02990198FFF7EAFC04000ED40198001901902D1B36
:204F40002100380002F0BAFA02988442E5D00098441B002D02D0280002F0BAFA002F02D078
:204F6000380002F03BFAC046200004B0F0BD0000FEB504000025180002F014FB002602F03E
:204F80001DFB0099091A8F1B002803D0402FF6D303208743002D0BD102988319019A390060
:204FA0002000FFF73DFD0500BD4200D10025E419F61900988642E2D1002D01D00020C04367
:204FC000FEBD0000FFB50024E443042102A802F0CBFA0421684602F0C7FA009803900002DE
:204FE000000A0090050002F0C3F906000098B04200D20600300002F0CDF907000DD1002D02
:2050000002D0280002F0BCFA002F02D0380002F0E5F9A9E7029800190290002D14D0B54208
:2050200001D2019500E0019601982D1A3B00039A01000298FFF79CFF0400E0D40198844295
:20504000E8D00024E443DAE7009CDFE730B5A9B0002404E021A8694609780155641C0121F3
:20506000684602F081FA68460078FF28F2D1220001A921A8FFF734FD0500A10001A802F008
:205080001DFA280029B030BD10B5AAB000240CE0042101A802F068FA22A86946097801556A
:2050A000A00002A9019A0A50641C0121684602F05BFA68460078FF28EAD1220002A922A87A
:2050C000FFF758FD2AB010BD0FB50020019014210291039004E06846017801A802F044FA2A
:2050E0000121684602F040FA68460078002806D1039A02990198FFF7D1FE04B000BD012166
:2051000000A8401C02F030FA684640780128E2D0022802D0032804D007E06846017802A87B
:20512000DCE76846017803A8D8E76846007802F027FAD5E730B591B004000221684602F039
:2051400013FA6846018801A802F00EFA68460088042803D301A804F091FF00E01E481F4955
:205160000860642C10D0652C11D06E2C12D06F2C13D0792C14D07A2C1CD07B2C1DD07C2C94
:205180001ED0822C1FD021E0FFF7AAFE1DE0FFF719FF1AE0FFF75AFF17E0FFF775FF14E03C
:2051A000012100A8801C02F0DFF968468078FFF72DFD0AE0FFF740FD07E0FFF71DFD04E001
:2051C000FFF700FD01E0FFF77FFF0500280002F0B1F911B030BDC046FF000003D80120000F
:2051E00008B4024B9C4608BC6047C0464813200010B504000E480078FF2809D105220D49C3
:205200000D4804F08BFF002804D001F079F810BD0028FAD0002C01D001F05AF801F060F815
:20522000002CF4D0142002F059FD01F055F810BD04FD1000ACAC100010FF1000F3B585B082
:2052400000240025022104A802F08EF96846008AC01DC01000900321484302F09BF8019083
:20526000009801990818029000980299081803900198002808D10098400002F081F90098EE
:2052800002F026F9062553E00099029802F06CF90099019802F086F902F090F90099091A3B
:2052A0000E1B002803D0FF2EF6DD3F208643F7000098814206D16846008AC01D4007400FCE
:2052C000C01F3F182D062D0E1FD12748007800280FD139000298001901F092F83B0003980E
:2052E0000219029801190198001901F011FB050012E0012810D13B0003980219029801198A
:205300000198001901F04CFCF1E7FF1DFA1000210398001904F022FF0698002804D13100EE
:205320000398001902F0EEF8A41900988442B3D10E480178002900D10570069800280ED15F
:205340006846007DCF2806D06846007DD52802D002F002F903E02806000E02F0DBF80198F1
:2053600002F03CF807B0F0BD870E20007C0E2000F0B588B00221684602F0F6F8022103A8E8
:2053800002F0F2F8022104A802F0EEF8022105A802F0EAF8022106A802F0E6F8684600880F
:2053A00003214843093001F0F5FF040068460088211801910D1868460188200002F0D4F8E1
:2053C00068460188019802F0CFF868460699418005998183039F008804990904090C6E1825
:2053E000C00002900299200001F00AF802F0F2FA00F06AFF00F070FF3800471E000410D096
:20540000029B2A002100019801F082FA30787178090201436846808B084069464988884273
:20542000EAD102F0FBFA68460188280002F046F8200001F0D3FF08B0F0BD0000F7B582B015
:205440006846808D69460F8E8E8E1418D80000900099039800F0D4FF012002F03FFC00F060
:2054600033FF00F039FFA64D28686946098D40180190009B049A0399029801F049FA2078E6
:205480006178090201433940B14203D001982968401AEED505B0F0BD70B5C0B0802464005F
:2054A0002100684602F060F821006A460B48030015781E782E40AE4207D1521C5B1C491E07
:2054C000F6D12200694600F067FF0020FFF790FE002002F01FF840B070BD000000FF1000E5
:2054E00070B5A1B0002600240421684602F03CF80BE0C00705D5300001F096FA01A9485173
:20550000641C761C009840080090A50000980028EFD1290001A801F0D1FF21B070BD000053
:2055200030B5A1B0002400250421684602F01CF8C04801AB0DE0D20706D50022D243022C59
:2055400000D202685A506D1C641C009949080091001DA900009A002AEDD101A801F0AEFF52
:2055600021B030BD10B5C0B0802464002100684601F0FAFF22006946024800F00DFF40B070
:2055800010BD000000FD1000F0B5A5B0012100A8801C01F0E9FF042103A801F0E5FF04212E
:2055A00004A801F0E1FF012100A8C01C01F0DCFF012102A801F0D8FF0221684601F0D4FFD3
:2055C0009E4C002069468978642902D0652948D059E069460988002914D101E0002911D496
:2055E00046490A88521C0A8069460A80002122000A3213886D462D88AB42EFD0491C103284
:205600000429F6D3002122000A3203E0491C103204290CD213886D462D88AB42F6D10029A0
:2056200005D40801201836490968C1602BE06946097A6A46D278049B039D26000A3603E080
:20564000401C103604281ED23788002FF8D10001201805604360027241726946098841816B
:20566000E1E769460988002223000A3303E0521C1033042A07D21D888D42F8D1002A02D4C8
:2056800011016118488105A801906846018801A804F0BEFC042101A804F0BAFC102101A898
:2056A00004F0B6FC042101A804F0B2FC0425216801A804F0B5FC616801A804F0B1FC217A26
:2056C00001A804F09FFC617A01A804F09BFC618901A804F09DFCE16801A804F0A1FC10349C
:2056E0006D1EE4D100F040FF010001A804F098FC4C2105A801F0E2FE25B0F0BD780E2000F6
:205700005C032000F0B581B041480168491C01600A2979D1002404603E490A681000012845
:2057200014DB3D4A904200D10120401C08603B49884214DB642104F02BFD002803D0002072
:2057400001F06EFB0BE001F079FB08E0002806D5521E0A603248824201D101F005FA00F0EA
:2057600003FF34492F4A9042086812D32E4A904214DA002802D14868401C486008680A3079
:20578000086000F02FFF00280AD1012001F048FB09E0002802D04868401C48600C60F0E751
:2057A000012001F04BFBFDF703F920480168491C01600A2928D1046001F030F91E48006892
:2057C00000901E4801000A3104220B88002B18D0009B891C0D68891E5B1B154DAB4210DBBF
:2057E0000B88002506000A3603E06D1C1036042D07D237889F42F8D1002D02D42B01C3187C
:205800005C811031521EE0D101F0EAFA01B0F0BD2C022000F0042000FFFFFF7FB302000083
:20582000F0D8FFFFD6060000005C26053002200088130000E40120005C032000EC012000C1
:2058400000B502F0C7F8002001F006FBF9E70000F0B594B00600F42E02D1FEF7FDFB41E3FB
:20586000F52E02D1FEF7FEFB3CE3F72E02D1FEF739FC37E3F82E02D1FEF742FC32E3C22EB8
:2058800002D1FFF74DFE2DE3EB2E02D102F0D4FD28E3FDF789F8CE2E01D0CF2E0BD10120EE
:2058A00001F06EFE002800D01CE300213006000EFFF7C4FC16E3D52E08D1012001F060FE34
:2058C000002800D00EE30121D520F1E70024D62E05D1E04D287801F01DFE2C7002E3012572
:2058E0002902701EFD2800D9FAE202A24000125A9744C04650043A042E046E04C802680478
:205900000A03AC0462056805F005EC05EC05EC05EC05EC05EC05EC05EC05EC05EC05EC05A6
:20592000EC05EC05EC05EC05EC05EC05EC05EC05EC05EC05EC05EC05EC05EC05EC05EC0557
:20594000EC05EC05EC05EC05EC05EC05EC05EC05EC05EC05EC05EC05EC05EC05EC05EC0537
:20596000EC05EC05EC05EC05EC05EC05EC05EC05EC05EC05EC05EC05EC05EC05EC05EC0517
:20598000EC05EC05EC05EC05EC05EC05EC05EC05EC05EC05EC05EC05EC05EC05EC05EC05F7
:2059A000EC05EC05EC05EC05EC05EC05EC05EC05EC05EC05EC05EC05EC05EC05EC05EC05D7
:2059C000EC05EC05EC05EC05EC05EC05EC05EC05EC05EC05EC05EC05EC05EC05EC05EC05B7
:2059E000EC05EC05EC05EC05EC05EC05EC05EC05EC05EC05EC05EC05EC05EC05EC05EC0597
:205A0000EC05EC05EC05EC05EC05EC05EC05EC05EC05EC05EC05EC05EC05EC05EC05EC0576
:205A2000EC05EC05EC05EC05EC05EC05EC05EC05EC05EC05EC05EC05EC05EC05EC05EC0556
:205A4000EC05EC05EC05EC05EC05EC05EC05EC05EC05EC05EC05EC05EC05EC05EC05EC0536
:205A6000EC05EC05EC05EC05EC05EC05EC05EC05EC051404A604EC056E05EC05EC05EC05B4
:205A800032052004420348034E035403FC01EC05EC0576037C03EC05EC050E04EC05EC05C6
:205AA000EC05EC05EC05EC05EC05F002F6025A037003EC05EC05EC05EC05EC05EC050203CC
:205AC0003C03820404025A02EC05EC058804EC05EC05FC02C80446044A04EC05EC05F00417
:205AE000EC05EC05EC05D404CE04EC05EC05DA0400213006000EDBE60121684601F034FD51
:205B0000290000A8401C01F02FFD022001F038FD002800D0E6E1684600780002694649789C
:205B20000143FF20801C81420AD04B48814207D04A48814204D0B0200001814202D002E02B
:205B4000474D00E00725280001F0F4FCCAE1012100A8401C01F008FD2900684601F004FD0C
:205B6000290003A801F000FD290003A8401C01F0FBFC6846007B00026946497B0143FF204A
:205B8000801C81420AD03448814207D03348814204D0B0200001814208D0A3E16846437B48
:205BA000027B01784078FFF7C5FA9BE16846437B027B01784078FCF713FE93E1022100A8A9
:205BC000801C01F0D1FC68464088C749884201D16846448068464088FA218900484300F042
:205BE000ADFD7FE100F074FB7CE100F075FB79E100F030FCA8E7C14801F060FC72E104AC21
:205C000000F0B2FC208000F0D3FCA07000F0D6FCE07000F0D9FC207100F0C2FC607100F0A0
:205C2000E1FCA07100F0D8FCE071082104A8E3E7FFF732FC56E100F039FD53E100F03CFDE4
:205C400050E100F03FFD4DE100F042FD4AE100F037FB47E17C0E2000010300000106000060
:205C6000FF03000000F030FB3CE1FFF781FB39E1022100A8801C01F077FC022106A801F0D1
:205C800073FC022107A801F06FFC022102A801F06BFC022101A801F067FC68464088032188
:205CA0004843093001F076FB04006846408825182E1868464188200001F056FC6846418870
:205CC000280001F051FC019B029A079906980004000C0904090C1204120C1B041B0C0FB479
:205CE00004A84388320021002800FFF7A7FB04A84188300001F0E2FB200001F06FFB04B078
:205D0000F0E001F035FB1FE704A800F07FFE062104A871E700F0E2FC00F050FC01F0FAFB58
:205D2000E0E000F0D5FA022001F0D8FF5DE700F0C7FA022001F0D2FF94E771485CE7FFF7B4
:205D400011FCCFE001A800F015FB040001980004000C01F0E7FB019920004DE700F0F0FA96
:205D6000C0E0042001F0DEFB604801F0DBFBE80201F0D8FBB6E004215D483DE72022002191
:205D80000CA804F0EBF95B490CA804F055F90CA80571202101F092FBA4E0FFF7A1FBA1E05D
:205DA0000121684601F0E0FB68460078002802D000F096FA96E000F0A3FA93E000F05EFAE9
:205DC00090E000F05DFA8DE0FEF7E6F98AE0042101A801F0C9FB042102A801F0C5FB0299C3
:205DE000019809E708A8046044608460C4600A264148099000F0B4FE002801D508950FE0DC
:205E000024180999884200D209900A99814200D20A90761EEED120000A2104F0B1F90B91C5
:205E2000102108A8B6E70121684601F09DFB0190002857D168460078FE2803D0FF2804D18F
:205E4000032004E02F48007801E000F025FA0190042101A8D0E6FFF797FB43E001F036F87D
:205E600040E00121684601F07FFB042101A801F07BFB042102A801F077FB019802990143E8
:205E800030D0029C01F074FAA04202D201F070FA0400200001F07EFA050001D1FFF7D0FCCE
:205EA000029EA64201D2370000E0270068460078642802D0652805D008E03900280001F029
:205EC00053FB03E03900280001F0F8FAF61BE8D10198401E0190E3D1280001F07FFA01E0D4
:205EE000FFF7AEFC14B0F0BDFFFF0000E32E0000B4AC1000BF7BFFB900CA9A3B00FF100072
:205F000000FD1000870E2000FCB589B007000E00129C159800251399C91DC9080591169998
:205F20004907490F0791002C3ED00091C108149A5118049101210722024091400906090E5D
:205F400002911698C00810990818019013E000F0D1FB04980078029908421ED1059B149AF9
:205F60001199109800F07AFC002812D100F0C2FB6D1C761E16D0009A39680198FBF064FB90
:205F80003F1D2300149A0A99099800F067FC0028DDD00020C0430BB0F0BD1798B6490968BE
:205FA000401AEED52800F6E70695079800900698002803D1109804901A9802E01998049046
:205FC0001B9802901898B04201D2039000E003960398361A1698C008049908180190039CAD
:205FE000009A39680198FBF02FFB3F1D009813994018C108019A511801914007400F00903B
:20600000641EEDD103981899884201D2029800E000200090139C0398444311980290E01D24
:20602000C0080590009800281AD0059A029904F03BF86007400F019010D0E00800990C182C
:206040000821200000F0DCF92078FF21019A9140884320700821200000F0D2F90098029085
:2060600000F048FB059B149A0299049800F0F6FB00288ED1069801214140069103982D1848
:20608000002E92D100F036FB8CE70000F1B577498D440024009401F06BF9099001F07AF99A
:2060A0000B900DA801F086FA0EA801F083FA03A801F080FA0FA801F07DFA10A801F07AFAA9
:2060C00008A801F077FA04A801F074FA0D98C01DC6080E98C01DC00802900398C01DC7082F
:2060E00002983018C0194500FF20801C854200D3B4E0290011A801F037FA08985E490968FB
:2061000040180890700011A908180C9002980C9908180A9002980A9908180590C01906904F
:20612000012001900298002826D180200001039904F026F801910498884200D20190019BAE
:20614000039A0699FFA8483003F01EFF019B039A059991A803F018FF01980499884205D2E3
:206160008022520091A9D1A803F09EFF91A80590FFA84830069003E0C1000A9800F040F9F6
:2061800001984743F900069800F03AF911A88519F100280000F034F9330051AA290011A885
:2061A00000F05CFB00F0A6FA04980790079885000998854200D3050029000B9801F0F2F9C9
:2061C000002601F0FBF9291A032291438F1B002801D0402FF5D30098002821D4244B6B44CB
:2061E000FFAAFF324932D1A901980FB40C9B149A139955A80FB40B9B0A9A0E990D980FB45A
:20620000169B189AB9088C46B0108100179840186146FFF779FE0CB00090002800D42418A8
:20622000F619AE42CDD10798A908401A0790BDD1104868440078002805D00098002800D4E5
:206240000094042107E00498844201D0012000E0002000900121684601F030F90B9801F03C
:20626000BDF8E920C0008544F0BDC046BCF8FFFF44060000440700005C032000002005E752
:2062800000B581B00121684601F06EF90120FFF7FDFE01B000BD000070B50400074D287853
:2062A0000600012803D1012C01D002F04FF9200000F084FC2C70300070BDC046870E20005F
:2062C00000B500F0A1F900BD00B500F0A3F900BD00B500F0A5F900BD00B500F0A9F900BDC0
:2062E00000B582B000F0B6F900206946088048808880C880012000F0BFFD02B000BD00006D
:2063000000B582B000F09CF900206946088048808880C880012000F0AFFD02B000BD000076
:2063200000B582B0684601210180FA21490041808180C1806946012000F09EFD02B000BDF4
:2063400000B5094800210160012001F0E3F8642001F0C4FC8120400300F03CF803480449F3
:20636000016000F001FC00BDF0042000400020002143341200B501000548064A1378002BEB
:2063800000D01000002901D070220A6000BDC0465020100070042000F0B504000D00160084
:2063A0000AE07700012F04DB002000F039FD7F1EFAD1002000F042FD320029002000FAF00B
:2063C00041FE32002900200003F0A8FE0028E8D1F0BD000030B5C0B0040080256D002A0047
:2063E000FF21684603F0BAFE2A0069462000FFF7D3FF40B030BD0000004B18474510200067
:2064000000B5C908114A1268114B9A421AD30E4A04290FD30378D35C03704378D35C4370DB
:206420008378D35C8370C378D35CC370001D091F0429EFD2002905D00378D35C0370401CF8
:20644000491EF9D100BDC04678AD100060022000701700003548006870470000F0B40420A6
:206460002E4908602E490022D2430A60EC23DB022C4C23602C4C2360754B1A609B4B1B4CBC
:206480001C609B4C1A4D2560874C1A4D25601A4D1A4E2E605B4D2D680226244FBC466F0A3E
:2064A0003840AF0B374007436D0F0120284038438000134D2858674638601D4802601148A4
:2064C000026098208002104A106008603103196020600E480E4901600E48FF2101600E4886
:2064E0007021016013480660F0BC704700021081936100089303100964F4FFFF008800204A
:20650000B8AC1000A4F4FFFFA0F4FFFF0480FDFF000B09031480FDFF1080FDFF10FCFFFF22
:2065200000F4FFFF70F4FFFF04F4FFFF5C02200060F4FFFF0080FDFF00B56C49002802D061
:20654000012803D000BD0220086000BD086000BD00B56749002802D0012803D000BD0220DC
:20656000086000BD086000BD10B5954CA078002805D1012001F0B2FBA0780028F9D02069C4
:2065800005494843054903F003FE0800642800D200200004000C10BDDC190000FF03000086
:2065A000184800680104890E012008407047000014480068410E0120084070471148006863
:2065C000810E0120084070470E4800680104090F01200840704700000A480068810D0120A8
:2065E0000840704700B506480068E62801DA012000BD04480068410D0120084000BD000042
:20660000480220003CF4FFFF384880214900016070470000364880214900016070470000E0
:20662000334880214903016030488021016070472E488021490301602D488021016070476E
:206640005F48002101700248802109060160704714F4FFFF30B55A4C2078002822D101208A
:2066600001F03CFBFA204000FAF0BCFD802000061E4908600C490860012001F02FFB002067
:20668000E07020626060208121000A3122001432032300250D801060121D891C5B1EF9D1A4
:2066A0000120207030BD000010F4FFFF0F48802189010160704700000D48802189010160BF
:2066C000704700000948802189020160704700000748802189020160704700008020C0017A
:2066E00002490860024908607047000034F4FFFF30F4FFFF00B5C04800688349884211D396
:20670000094800680028FBD1804800688005FBD59820800205490860BB49802292010A60B4
:2067200003490860002000BD0441FDFF00F4FFFF10F4FFFFB04800687047000070B5040053
:206740001F4DAC6230D00122AE4B00261748184909780129A96A0CD1164CA14207D203F011
:206760000FFD891E196001291EDA1A6070BD1E6070BD03F005FD0A3900D500211960B820FA
:206780008002844202D3A448112101E019210A48E9620A4B0019401E210003F0F1FC1970B0
:2067A0001878000202432A6370BDC046808D5B00870E200000D4300060E316009800200010
:2067C00038022000FFB500980678019805780027082480208002F10701D5894900E08A49B7
:2067E0000860E80701D5864800E087488021890101608548490001606D0876087F088148A9
:206800000068002801D0FAF0EFFC7C480068C00402D538008027074379488021C9010160C5
:2068200078480068002801D0FAF0DEFC641ED0D10298077074488021890101600198401C02
:2068400001900098401C00900298401C02900398401E0390B7D104B0F0BD0000F0B504007D
:206860000D001E00BC480169E62901DA0520F0BD806A204F204BB8218902884210D33100BD
:20688000100003B43A0029002000FAF02FFC1B4806601B48802149000160002002B0F0BDA3
:2068A0001949884216D33100100003B43A0029002000FAF01BFC802080001449114A02B0BD
:2068C0002B7813606D1C0B680342FCD0761EF7D10020F0BD002805D1F3002900200000F042
:2068E00059FAF0BD330029002000FFF76BFF0020F0BDC0460000FEFF0040FDFF0C01FEFFA6
:206900002001FEFF0C00FEFF701700001000FEFFF4B582B004000D001E0036480068E628BE
:2069200001DA052063E0F7080AD03B002000FFF795FF0090FFF7DEFE0098002856D101E02C
:20694000002000907607760F50D0ED19E4190298C019029028480068002807D13300029AB6
:206960002900200000F016FA00903FE06846868024782E788588002780208002E10701D515
:206980001F4900E020490860F00701D51C4800E01D488021890101601B4849000160760851
:2069A00064087F0817480068002801D0FAF01CFC12480068C00402D5380080270743104844
:2069C0008021C90101600F480068002801D0FAF00BFC6D1ED0D1029808216A469288891AE6
:2069E000CF4007700848802189010160009803B0F0BD000048022000600220003CF4FFFF23
:206A000030F4FFFF3402200034F4FFFF024901600421818070470000006CDC02014858491B
:206A20000160704740FDFFFF00B54B490C281DD801A2125C9744C0460E12161C223434348F
:206A40003434282C3000087800BDC87800BD0420085E00BD0620085E00BD0820085E00BD35
:206A6000488900BD888900BDC88900BD0020C04300BD000070B53848816B314A12688B18A3
:206A80008363446B641C446300220121082C04D1DB10036142638263817002240378002B57
:206AA0004AD0036A5B1C0362264D2D68264E3668AD1B264E7543AD1285800626865FAE42A0
:206AC00000DAC580642B04DB0823C35EAB4200DA05811F4B9D420EDB4269521C42614389D6
:206AE000934200D24281022A09D3C170FFF708FCFFF716FC20E0426116498D420ADB826950
:206B0000521C82618189914200D282810A2A06D3C470EBE78261FF2192318D420BDBC269B9
:206B2000521CC261C189914200D2C281282A03D30321C170DAE7C2610848046070BDC0464A
:206B40004080FDFF4480FDFF4880FDFFC8190000B90B0000E9030000380220000080FDFF8E
:206B600000B5FAF0A9FB00BD00B500F033FF01F06FFB024802490160FEE7C04600FDFFFF07
:206B8000010000A502489021490001607047C04614FCFFFF3E489021490001607047000047
:206BA00010B5040008000449096802B4210000F0F9F8002001B010BD3402200010B55F4B2B
:206BC000802292001149104C002804D001280AD002280ED010BD1C60882080020860500198
:206BE00018600A6010BD1A60C020C00108600C6010BD5D4804605B481023036098208002AE
:206C000008600A6010BDC0461000000834F4FFFF30B5194C21603D4D2A603D4A13601C4854
:206C20004021016020201B4908601B4908601F4804210160C8214900016010481049016028
:206C4000104B11482168C90003F09AFA491C480818600E480021C94301602A482968016032
:206C600029481168016000202A4908602A49086023480121016030BD740220000400FCFF83
:206C8000C00808002000FCFF0080B6050C00FCFF10FCFFFF04F4FFFF70F4FFFF03482021D9
:206CA0000160174802210160704700000000FCFF144A1268026014480068086070470000C1
:206CC00030B5040000F086FE0D480221016001600C490B680C49A34201D2E21A0AE00B4A0D
:206CE0001268D31A0A4D2D685B190B6009490A600949A21A0A600121016000F061FE30BD6F
:206D00002001FCFF0001FCFF0401FCFF780220007C0220001001FCFF1401FCFF0048704708
:206D2000D8AC1000802040050349086003490860034908607047000000F4FFFF30F4FFFFF3
:206D400010F4FFFF80204005064908600649086070470000802040050249086002490860DC
:206D60007047000060F4FFFF14F4FFFF00B5054800681F2188430449884201D1034800BD9E
:206D8000034800BD40F2FFFF40090D27FFFF2000FF3F200008B4024B9C4608BC6047C04666
:206DA000F011200008B4024B9C4608BC6047C0463C13200000B50A214143434A51188A788B
:206DC000002A01D0497800E00978002902D0FFF7B3FB00BDFFF7BCFB00BD00007047000019
:206DE00060B501250D4E3088002811D0401E308000040DD1F01E0178002901D0B28800E0B1
:206E0000728801234B40037032802800FFF7D2FF6D1E0A3E002DE6D560BDC0468E02200027
:206E200000B50A214143284A511801220A708978002901D1FFF780FB00BD000000B50A216C
:206E40004143214A511800220A708978002901D1FFF77EFB00BD000000B50A2141431A4A4E
:206E600051180A78012353400B708978002901D1FFF7A0FF00BD000070B5022823DA0A222F
:206E80004243114B9A180B8893708B88D380CB881381CC8801250023002C02D19380557008
:206EA0000BE08E88002E01D1938005E04E88002E01D09680F3E7948053700988002900D1B2
:206EC0009380FFF777FF70BD8002200030B583B00221684600F048FB00241BE0022100A85E
:206EE000801C00F041FB022101A800F03DFB01AD0221A81C00F038FB0221281D00F034FB97
:206F00000221A81D00F030FB01A968464088FFF7B3FF641C684600888442DFDB03B030BDD0
:206F2000F3B585B0B2480168CB104C07640F01940824019D641BA24201DA009200E00094CD
:206F40000124009DAC40641E6A4D2D68EE180296674E36680496F6180396019E002E17D0CF
:206F6000039E40B43678B44601AE377D2740029EB7406646374340BC3770029EB446367862
:206F80006F463F7E3C40019FBC40344366460BE0039FBC466E46377D26003E4067463E704E
:206FA000029E6F463F7E3C403470009C121B0919002A0CD05B1C049C6E46367D009F3E4112
:206FC000E6546C46247E009E3441EC548918016007B0F0BD10B50400082C07DB0822FF2141
:206FE000002000F0D7F8083C082CF7DA012C06DB01220121002000F0CDF8641EF6E710BD15
:20700000F0B581B004000E001500002E45D078480068002804D1002B02D0012000F06CF899
:207020001F480068401B871B04220021032000F0B1F8002F02D03800FFF7CCFF6C4800686B
:20704000009008E000203A0021780006000E00F0A1F8641CF61B012E0CDB082E01DA370039
:2070600000E00827002DEDD1092EEBDA0120711E8840E8E7002D09D0022D02DB681EFFF745
:20708000A9FF01220121080000F084F801220021012000F07FF8009800E0002001B0F0BDCD
:2070A00048002000F0B5524C216800291CD0104D28680E4A12780F4E354F002A0AD10722A9
:2070C0009143FFF79DF923683A6829683068FFF71FFC07E0012A05D10B003A6801003068BB
:2070E000FFF75EFD00202060F0BDC046870E2000AC022000A802200010B5040004E00122CF
:207100000021002000F046F82000441E0028F6D110BD000036480168C91D07229143016097
:20712000C0E70000BEE7000010B50400FFF7BAFFE01017490968091808786207520F08D087
:20714000D040030048780821891A884018430006000E10BD10B50400FFF7A4FFE0100C49E5
:207160000968091808784A7812020243887803041343C91C0878000618436207520F06D01F
:20718000D040030048782021891A8840184310BDA4022000F0B581B004000D001600134F23
:2071A0003878002808D0062200211F20FFF7B8FEFFF7B0FF002038700D4800680090012E02
:2071C00010DB092E01DB082700E037003A002906090E2006000EFFF7A3FEF61B240A2D0AAA
:2071E000012EEEDA009801B0F0BDC0467D0E2000A00220000023014A126801E798022000A5
:20720000F0B581B0002901D100203EE03A4A15680E0004003D480068471B7F1E032200211A
:207220000120FFF7B7FF002F04D03A0000210020FFF7B0FF16480068009008E000203A00C6
:2072400021780006000EFFF7A5FF641CF61B012E0CDB082E01DA370000E00827002DEDD1FE
:20726000092EEBDA0120711E8840E8E7002D06D02A00002101206D1EA840FFF78BFF012246
:2072800000210120FFF786FF009801B0F0BD0000A002200010B504000320604300F07AF888
:2072A00000280DD01C4908601D4902190A601B49620082180A600C490C60164900220A609B
:2072C00010BD000010B5144C206800280BD000F085F8002020601249086010490860024955
:2072E00008600C49086010BD9C022000024A11600249086070470000940220009802200047
:20730000024A106002480160704700004400200048002000A0022000A4022000AC0220002D
:20732000A802200000B50022426001602A490A68002A01D1086000BD0A0000E01A1D136807
:20734000002B01D09842F9D24360106008680028F1D000E0080041680029ECD002688318A5
:207360008B42F7D14B684360096851180160F2E700B5002018490968002909D00A68904221
:2073800000D2100049680029F8D1002800D0083800BD000010B501000020C91D07229143AA
:2073A00008310D4A00E01A1D1368002B13D01C68A14208D218005B1813600268521A1A600E
:2073C00042685A6003E0EED118005B681360002801D00160083010BDB002200000B500284B
:2073E00003D008380168FFF79DFF00BDCA1D07218A430832083801680260891A801891E7EE
:2074000010B504002068FFF7E9FF0020206010BD0722914386E7000010B581B0204CFFF70E
:20742000A5FC011B491C2000FFF7F2FFFFF716F81C48FFF783F90120FDF7DAFEFFF794F8DA
:20744000FFF7CCFC0020FFF7EBFC00F0C7F8164C1CE0FFF7E5FC01202060FFF793FB6846BA
:2074600000F0DAF800280BD1FFF794FB0020C04320600020FFF7E2FC68460078FEF7E8F92E
:2074800000F014F80028E4D000F0B8F800F0C0F80028F5D1FFF7E0FC322000F01FFCF5E7D3
:2074A000E0192000204E0000F004200000B574480068806802F028FE00BD000000B50A00DC
:2074C000024304D06E4A1268926902F055FD00BD70B588B00400684600212022121F8150F1
:2074E000FCD1674D212C01D3202600E02600310068462A68926902F03FFDA41BF2D108B0CA
:2075000070BD000000B55E4A1268D26902F034FD00BD000001B501216846FFF7CFFF01B051
:2075200000BD000001B502216846FFF7C7FF01B000BD000001B504216846FFF7BFFF01B0EF
:2075400000BD000001B5042168464D4A1268126A02F012FD01B000BD00B549480068406A91
:2075600002F0D2FD00BD000000B5002901D1002000BD434A1268D26802F0FEFC00BD000016
:2075800030B588B00400212C01D3202500E0250029006846FFF7E8FF002801D1641BF2D16F
:2075A00008B030BD00B5364A1268126902F0E4FC00BD0000002101600221D5E700B53048DF
:2075C0000068006802F0A0FD00BD000000B52C480068406802F098FD00BD000000B52948EC
:2075E00000F0F4FB00F078F825482749016000BD00B5244800F01EFC00BD000000B500F0C4
:20760000CFF81F480068406902F07EFD00BD000000B500F0B7F900BD70B581B00400184D30
:207620002868806802F070FD002801D0FFF7E6FF00F0B4F9134E00F0A5F9002804D10221F3
:20764000300000F031FC06E00021684600F080F9300000F011FC00F095F90028EBD000F041
:207660008DF90128E7DB0848286001212000FFF77BFF040000F09AF9200001B070BD00008A
:20768000B4022000B80220000CAD100000B5FFF7AFFF00BD00B501F0FDFE8007800F02287A
:2076A00001D0FFF7A5FF00BD014800887047000094002000374800887047000001480068F7
:2076C000704700005C0020000148006870470000600020002B48704710B581B00A22294BCF
:2076E00029480078012802D0022812D013E0274804680A3320000A2102F042FD303018702B
:2077000020000A2102F03CFD0C005B1E521EF1D109E01F48ECE716480078042803D21D49DC
:20772000F7328018088001F02DFC6C46002001B4002340220221012001F098FB2070402022
:2077400001B40C4B02000221002001F08FFB607002A800F067FF01F031FC074800F082FFAF
:2077600000231A000549064801F05CFE03B010BD00FD1000D40220008D7610009576100034
:20778000C40220005000200001FD100000FF100008FD1000960020007348007870470000C1
:2077A000714800210170704700B5FFF7CBFA0A2000F094FAFFF7B6FA00BD0000F2B581B074
:2077C00069490978002947D10400019E4F4D2F68002F1FD04020C01B864201D2009600E0F5
:2077E0000090009A21002F48C01902F05DFC00983F182418361A402F0CD16F480368002298
:207800004021284800F0F8FE402802D05648012101700027B009800100900FD0664803685D
:2078200000220099200000F0E7FE0099884202D04D480121017000982418361A002E05D014
:2078400032002100174802F02FFC37002F6030480168019A8918016002B0F0BDF0B52C4C99
:20786000206800281CD0404D2978002918D1274E3168002700290CD04F480368012209487C
:2078800000F0BAFE3168884201D001202870376005E0810603D1400501D000F0A3FE27604E
:2078A000F0BD00001403200070B504000D002E4E307800280CD1FFF7D1FF3F4803680122AA
:2078C0002900200000F098FEA84201D00120307070BD000030B505000C002348007800282F
:2078E00012D10A480068002801D0FFF7B7FF2100280000F055FE0648A10602D00021016071
:2079000030BD01680919016030BD00005403200058032000F0B504000D000026F643124F39
:207920003878002801D03000F0BD23480268200000F06EFEA84208D02A000021200002F051
:207940000DFC012038703000F0BD0020F0BD000000B5054A1278002A02D00020C04300BD41
:2079600000F016FE00BD00007E0E200000B500F02FFE00BD00B500F023FE00BD00B500F0E3
:2079800019FE00BD00B501F085FD8007800F022801D1012000BD002000BD00000648074980
:2079A00002680A6000210160704700000248034909680160704700004C002000C00220004D
:2079C0007847C04600C00FE180C0CCE30CF021E11EFF2FE17847C04600C00FE180C08CE3F4
:2079E0000CF021E11EFF2FE17847C04613F021E31EFF2FE17847C04693F021E31EFF2FE1EA
:207A000005480178491E01707047000002480178491C0170704700006003200000B503483E
:207A20000078002801D1FFF7CBFF00BD6103200010B5FFF7CFFFA74C2078401E20700006CB
:207A400005D189480078002801D000F04DF96078002801D1FFF7B4FF10BD000070B5816882
:207A60000024002906D00A684968002A00D051600A608460417B8907890F4173954D14D168
:207A800077490A68002A16D108602878002807D101202870FFF794FF00F026F92C7004E0CA
:207AA0007148017802220A4302706878002801D1FFF786FF70BD137B067BB342E4D38242B0
:207AC000F3D1E2E730B50400207B374900E011000A68002A02D0157BA842F8D322600C6083
:207AE000607B002804D1FFF775FF2000FFF7B6FF30BD0000F0B5FFF76DFF5B480178FE2249
:207B00000A400270574C774D2868FA21090140182060234E234F0EE0386001683160002131
:207B2000017438688160FFF74BFF3868406802F0EBFAFFF74FFF3068002806D081682A689B
:207B4000891A0129E8DB80682060FFF739FF1648066807E070692168411A00D52060FFF744
:207B60002FFF3668002E1AD0FFF734FF3C480168002904D0317B0068007B81420FD3707BEF
:207B80004007ECD570692968401A0128E2DA3000FFF764FFFFF71EFF707B0028DAD1F0BD2D
:207BA000700320007403200064032000F0B5494C00206070FFF71EFF294D05E0306828605C
:207BC000FFF712FFFFF716FF2E68002E20D0777B38001DD0780711D5706942490968411A33
:207BE000012906DA3000FFF739FF707B002805D10EE01C490A68821A00D50860FB20384003
:207C00001028DBD1B06880684068407B0028D5D115480178C90706D5FFF7E6FEFFF76AFF95
:207C2000FFF7E8FEF4E70178FD220A4002702A482968002909D02968497B0029296802D053
:207C4000896889684968016006E0016000202070FFF7CAFE00F0C6FAF0BC01BC004700001B
:207C60006C032000640020007F0E200010B5194C2078401C207000F037F82078401E2070F1
:207C80006078002801D1FFF79BFE10BD00B500F02FF81048012101704078002801D1FFF757
:207CA0008FFE00BD10B504000A480078002806D0FFF786FE0B480168091B09D5FBE7FFF7D9
:207CC00089FE05480068446104214173FFF7CEFF10BD000060032000680320000149096891
:207CE0004018DFE75C032000004B1847787F1000004B184758801000F2B5040015001E00C6
:207D0000069F1C22002102F029FA0C480178491C0170684600782073F0192C380321884392
:207D20000021016006494162856260602000FFF7C9FEFFF77DFE01B0F0BDC04660032000F3
:207D4000687F100070B584B004000D00029401940B4E30680390FFF73DFE2068009068461C
:207D600020600098002801D06946416030686946816030684573FFF779FF04B070BDC046D5
:207D800068032000F0B584B004000D001600029401940D4F38680390FFF71CFE2068009076
:207DA000684620600098002801D06946416038684661386869468160386804212943417358
:207DC000FFF754FF04B0F0BD6803200000B50822002102F0C3F900BD30B505000C4C207829
:207DE000401C2070FFF7F6FD6078401C6070280000F020F8280000F00DF86078401E607057
:207E0000000601D1FFF7DCFDFFF712FE30BDC0466003200010B50400FFF7DCFD00202071F6
:207E200003480078002801D1FFF7CAFD10BDC0466103200030B50500FFF7CCFD0D4C607897
:207E4000401C6070286800280AD02078401C207000202871280000F073F8FFF7E9FD01E0E7
:207E6000012028716078401E6070000601D1FFF7A7FD30BD6003200010B50400FFF7AAFDFA
:207E80002079002804D148212000FFF75BFF10BD0020207103480078002801D1FFF790FDB5
:207EA00010BDC04661032000F0B504000E00FFF791FD114D28688619104F2079002811D1A1
:207EC000320048212000FFF75DFFFFF783FD2868301A012806DA7878002801D1FFF770FDEF
:207EE0000120F0BD002020717878002801D1FFF767FD0020F0BDC0465C03200060032000EA
:207F000000B5FFF767FD0A480168491C016009480068081A04D40848017801220A43027073
:207F200006480078002801D1FFF74AFD00BDC0465C032000640020007F0E2000610320004D
:207F400010B5040002E0C068FFF788FDFFF742FD20680028F7D103480078002801D1FFF773
:207F60002FFD10BD610320001FF021E30400A0E10040BDE81EFF2FE1F0009FE5003090E5C1
:207F8000F84F2DE9E8009FE5001090E504D081E513F021E3DCD09FE5DC009FE50FE0A0E152
:207FA00010FF2FE19FF021E3C4009FE5001090E504D091E5F84FBDE8B0009FE5003080E543
:207FC0001EFF2FE100402DE9B0009FE50FE0A0E110FF2FE10040BDE8A4009FE590109FE52A
:207FE000001091E5000051E398109F051320A0030600000A001090E5182010E59FF021E350
:2080000006002DE993F021E37C109FE51F20A0E3001080E5182000E51EFF2FE10F502DE9B7
:20802000D4FFFFEB64009FE50FE0A0E110FF2FE118208DE292F021E30300B2E801F06FE101
:2080400000E0A0E19FF021E30F50BDE808D08DE292F021E304F05EE2F05F2DE90D00A0E134
:2080600093F021E300D0A0E1F05FBDE81EFF2FE16003200068032000A0192000AD7B1000E8
:208080000D7A1000DC192000987F100020801000017A1000704700007047000070470000AD
:2080A00000B504480068FEF7E5FCFDF72BFBFFF727FF00BD38FDFFFF70B5294829490160F2
:2080C00029482A4908609F21C943294A0A602949294A0A60294A1168C907FCD52849294BEA
:2080E0000B600423042411682142FCD0082114680C42FBD0244C25681C26B5432B43236038
:20810000082615683542FCD003251D432560082413682342FCD00022D2431C4B1A601C4B0D
:208120001A603B4A1B4B13601B4A1C4B13601C4A1F231C4C1460121D5B1EFBD11A4A0023A9
:208140001360491EFCD119490A68194B13400B6018490860FEF7FEFD012070BC02BC08476F
:2081600044FDFFFF0062FF0F010000A540FDFFFF0001480020FCFFFF0140000068FCFFFF69
:208180002CFCFFFF051C191030FCFFFF24F1FFFF28F1FFFF9580100034F1FFFF9D801000A6
:2081A00084F0FFFF9980100030F1FFFF20FDFFFFFFFFFCFF08FDFFFF00B5FFF70BFC0648EE
:2081C000064901600649012000F014F8012000F021F8FFF723FC00BD30FDFFFFB20B00039C
:2081E000A180100000B5024801210160FDE7C04604FCFFFF30B505000C00FFF7EBFBA8006A
:208200000349081805680460FFF708FC280030BD80F0FFFF10B50400FFF7DCFB03480121A1
:20822000A1400160FFF7FAFB10BD000020F1FFFF10B50100054A137818008B4205D00121B9
:20824000FF24E44321605940117010BD800E20000020EDE700B5402281214903D00301F001
:2082600023FF0120FFF7E4FF00BD0000F1B585B00026BD4D2868002806D102960396082131
:2082800002A8FFF71BF95CE004A901A8FEF710FD0198A968441A05D10498002805D1EC68CA
:2082A000012602E001D5E86824180598844200D20594029605980390082102A8FFF7FEF8FE
:2082C0000598002822D0A8680199884221D369680C1A05998C4200D30C00260013D0310003
:2082E000FFF710F9FFF772F9371AFBD0A868C019A8606968884201D32868A860A868FEF705
:20830000DFFCF61BEED10598001B05900598002815D0059C2100A868FFF7F4F8FFF756F9C2
:20832000261AFBD0A8688019A8606968884201D32868A860A868FEF7C3FCA41BEED1FFF742
:208340000BF906B0F0BD000070B581B005E06846017814342000FFF7DDFA01216846FFF759
:20836000D9FA794C6846007800282CD16069FEF7D5FC02001068516801F002FFA06981429A
:2083800000D2A1611068916801F0FAFEA069884200D2A16120680025002806D0E168226989
:2083A000914237D0FFF71AF825602069002826D1204EFEF7DDFF80190640802080008642A8
:2083C0001CDAED4330E0012100A8401CFFF7A2FA684640780128BAD0022802D0042804D09A
:2083E00007E0684601781834B4E7684601781034B0E768460078FFF7C3F8AEE7266120690A
:20840000FEF7C8FF20602069E060216808186060002909D0FEF742FC23692268A1696069D0
:20842000FEF7F6FB2068A0602800FFF783F801B070BDC04600FEFFFF30B582B0012100A874
:20844000801CFFF767FA00246846807866281FD1019403E0017801A8FFF75CFA012168462B
:20846000FFF758FA68460078002803D10198FFF7FDFE4BE0012100A8401CFFF74BFA6846CE
:20848000407803286846E5D00078FFF779F8E5E768468078642804D065280ED06E2820D0F4
:2084A00034E0FFF751FF31E0012100A8401CFFF731FA68460078FFF763F801216846FFF7CD
:2084C00029FA684600780028EED11F4D2868002805D0FEF7E3FB2868FEF780FF2C600020F0
:2084E00012E0019403E0017801A8FFF713FA01216846FFF70FFA68460078002808D101985E
:20850000002813D00020C043FFF714F802B030BD012100A8401CFFF7FDF9684640780128EB
:208520006846E0D00078FFF72BF8E0E71C20FFF709F80198FFF706F80198FEF7EFFB142118
:20854000FEF7BCFFE2E700006800200010B5064C2068002806D0FEF7A1FB2068FEF73EFF32
:208560000020206010BD000068002000D2F021E30CD09FE5DFF021E308D09FE508009FE525
:2085800010FF2FE1E0192000A01920003C21100000B50A0001003748007800F093FD00BD69
:2085A00000B500230A0001002D48007800F09EFD00BD000000B52F48007800F09FFF00BDB4
:2085C000274800782821484305490818C0687047284800782821484301490818C06870478E
:2085E0008403200000B50123002201211C48007800F0C0FD00BD000000B508B413000A00E3
:2086000001001748007800F0D7FD01B000BD000000B513000A0001001648007800F042FD78
:2086200000BD000010B5040000F0A0FF142148430A4908180830FF218170C17001710121E4
:2086400022789140012263789A400A4302800448217801706178417010BDC046FC03200036
:20866000810E200000B501000248007800F0A4FF00BD0000820E200000B5FEF753FB00BD1E
:2086800000B5024800F0CAFE00BDC04634AD100004490860802000010349086003490860B1
:2086A0007047C046ACF0FFFF28F1FFFF20F1FFFF00B58000764BC018102A23DB03780B7041
:2086C00003784B7003788B700378CB7003780B7103784B7103788B710378CB7103780B72E4
:2086E00003784B7203788B720378CB7203780B7303784B7303788B730378CB731031103A23
:20870000102ADBDA002A04D003780B70491C521EFAD100BD30B580005D4BC01803230424E6
:2087200003250D40641B23409A4200D21300002B05D0D21A0C780470491C5B1EFAD1130978
:2087400023D00C680470250A0570250C0570240E04704C680470250A0570250C0570240EAA
:2087600004708C680470250A0570250C0570240E0470CC680470250A0570250C0570240E09
:2087800004701031103A5B1EDBD193080BD00C680470250A0570250C0570240E0470091D41
:2087A000121F5B1EF3D1002A04D00B780370491C521EFAD130BD0000F0B584B0BD4C25685B
:2087C000E80708D52068012188438C4901432160002000F0E1FDC14EA80728D5206840014C
:2087E000400D0090002700280AD009280FD2020001A90020FFF75CFF009A01A9380004E0E4
:2088000068460773002203A9100000F023FD206880218843B249014321603770206802213C
:20882000884377490143216073488760C760082768071FD53078002801D0401C307001A847
:208840000821134A13780370401C491EFAD168460079000605D520680B490143216001203D
:20886000307020680421884308490143216001A801F0F0FA3D4204D02068B8436149014382
:20888000216004B0F0BDC046CF8000004B8000005000FBFFF0B592B00500A8008549405892
:2088A0008026400500D535432806000E00F02CFB0400354241D0282148434F490E186D069C
:2088C0006D0EA8007B4940180168012291434B4A0A43026000219E4AF368002B02D1B37927
:2088E000002B1DD003681A4302607175F068002803D1B079002800D0B1713788F068B842A8
:2089000000D2F7683A00B1682800FFF703FF01207075F068C01BF060B068C019B06050E0F9
:20892000737D002B04D003681A430260717548E0B160200000F030FD43E0A8005D494018F9
:208940000190009000684001460D3100200000F059FC070000D102AF00980068800604D47D
:20896000320039002800FFF7A3FEA000524908180099096842220A40402A01D101210160FB
:2089800002680121514001600198016803D0022291431B4A02E040229143164A0A43026000
:2089A0000098006880060CD402A8874205D1320002A9200000F04EFC03E03100200000F0AD
:2089C0002DFC6806C00D3B494018016809070FD50168082291430B4A0A430260AA49095D36
:2089E000002905D10168202291433D4A0A43026012B0F0BD0F800000840320004E80000050
:208A00004D80000047800000F0B543E0254804600E2525400126002D0AD00127B7403D42C5
:208A200003D03000FFF736FFBD43761C042EF2D31D4804422ED0E00701D5FFF7BDFEE00484
:208A400020D5C5480021C94301600021016019480168802212020A4302600C220021164828
:208A600001F07CFB03220021874801F077FB9C4801680F220A4302608548FF21891C0160F6
:208A800000F0ECFCE00501D500F008FDA00501D500F00AFD05480468054800680440B5D1A4
:208AA000F0BDC0462000FBFF011300001800FBFF1C00FBFF3000FBFF780320000748002178
:208AC00001707448016880229143054A0A43026001686E4A0A43026070470000830E200054
:208AE0004F80000000B507498022520002430A60A549002804D00868032202430A6000BD14
:208B0000086000BD0800FBFF00B500F019FA7449012282400A6000BD00B500F011FA5C4958
:208B2000012282400A6000BD10B5282358438B4B181840798406A40E2000FFF7EBFDA000E5
:208B4000544940180168024A0A43026010BD00005F80000000B5FFF78FFD00BD00B54179AD
:208B60000A0602D58022D20000E000220079012804D0022806D0032808D00BE01000802282
:208B8000520006E010008022920002E01000C022920002438806000E3E4980231B02134375
:208BA00043507948016802220A43026000BD0000F0B5060003D1002000F0B2FBF0BD282037
:208BC000704366490C18300000F0BAF905072D0F2788E068B84200D2E7683A00A16830006F
:208BE000FFF798FDE068C01BE060A068C119A160A800284A80180268124B134303602088CA
:208C00000600E268B24200D2E068002804D1A079002811D00020A071E068B04200D2E6684C
:208C200032002800FFF776FD01206075E068801BE060A0688019A06015480121A9400160EE
:208C4000F0BD00005F80000010B50C0000F078F94006400E0C4A230014540BD081000D4A2E
:208C600089180A68094B13430B600949012282400A6010BD800007494018016820229143B7
:208C8000054A0A43026010BD840E20006F8000001000FBFF3000FBFF4F80000070470000AE
:208CA0007047000000B500F0A5FC0948FFF7F0FC0848802101600848090101600848002106
:208CC000C943016005480021016000F089FC00BD098A100000FCFFFF10FCFFFF7400FBFF11
:208CE0001400FBFF30B50F4A13000020521C1C78002C09D1147801258D402C4204D001210A
:208D000019700006000E30BD1B1D401C121D0428EDD3FF2030BD000080000249081840885B
:208D200070470000840020000020704710B5040000F006F94006400E0749012282400A6016
:208D40000A68012383409A430A602820444303480019FFF703FF10BD2800FBFF84032000B2
:208D600000B500280DD1084809780029016803D002220A43026002E00222914301600020D4
:208D800000BD0020C04300BD0400FBFFF3B514001D000026F6436846007828214843864937
:208DA0000F18387C012840D000F024FCBC4800788007800F022836D1002C0DD02200019907
:208DC0003800183000F012F90600A41B019880190190002C03D126E0386A002823D1019833
:208DE000B860FC606846007811490968C96A01F08DF9002D16D0684600780799002902D090
:208E000000F012FC01E000F007FCF879002803D03019F968461A06E0F868002802D00026A4
:208E2000F64300E0361900F0DBFB300002B0F0BD1C042000F0B504000D001600282060437E
:208E40005D490F1800F0D6FBB868002809D0002E04D03100200000F0E7FB02E0200000F04C
:208E6000DBFB00F0BDFBF868281AF0BDFEB582B004005D4D286A00900020019028780328F4
:208E80003FD2282148434C490E186846017A2000009A526801F070F8070032D0FF2830D00C
:208EA00028220021300001F059F9E101394371716846007A307138000099496901F026F938
:208EC0000700002C03D10A98B84200D2070000F039FB0206120E6846017A380000F014FB6A
:208EE000040002D1022000F0A9FB34800498B0610A98F06168468089708028780190401C5D
:208F00002870019805B0F0BD10B5010000200B4A1278002A0AD0084B1C788C4202D1000667
:208F2000000E10BD401C28339042F5DB032000F085FBFF2010BDC04689032000FC032000AD
:208F4000282148431C49081840797047544800784108012008407047F0B5234C256A012601
:208F6000074F08E03800A96801F0D0F8E86801F0CBF8761C283720788642F3DBF0BDC046DB
:208F8000AC03200030B5184C2C220021200001F0E5F801202070084D78220021280001F082
:208FA000DDF8FFF76DFB0020216A496901F0AEF8288000F00BFB30BD8403200030B50A4C1D
:208FC000256A286801F0A0F8FFF7C6FF2A6C100004D021002431012000F0CEFF1020E071DF
:208FE000286901F091F830BDFC032000F2B50400150000261FE0E068411862688A4200D26C
:2090000011000F1AAF4200D32F003A0021680918009801F049F8ED1BA068C01BA060F6197B
:209020000098C0190090E068C019E0606168884201D10020E060A168002D01D00029DAD12E
:20904000002901D10020E060300001B0F0BD0000F0B504000D00160017E0E2681018884228
:2090600000D3401A8219914200D20A00171AB74200D337003A0029002368181801F014F82A
:20908000F61BA068C019A060ED19002E06D0A06861680A1AE1D1012000F0D0FAF0BD0000A5
:2090A0000304200030B504000020554D2D78AD07AD0F022D05D108B401232000FFF766FE6A
:2090C00001B030BD00B5002308B4FFF75FFE01B000BD000000B5914B9860D9609A710020B0
:2090E000AC490968096B01F011F800BDF2B5040015001F00002C05D041480078800701D4A2
:20910000002035E02820604384490E18307C0028F6D13079022806D13088401E284001D1A7
:20912000680500D1002700F065FAB06800280CD0F16840180099884204D1F0684019F06075
:20914000B7710CE0200000F067FA0098B060F560B77120008F490968096B00F0D7FF00F0D2
:209160003FFAF068281A03D1B179002900D0012001B0F0BD70B5040015000020204E327830
:209180009207920F022A15D12A002000FFF7AEFF291A727F002A05D105002000FFF74AFEFF
:2091A000281870BD012905DB050000222000FFF741FE281870BD0000F0B504001500059EEE
:2091C00000200F4F3A789207920F022A16D12A002000FFF78BFF291A7A7F002A06D1050006
:2091E00032002000FFF726FE2818F0BD012905DB050032002000FFF71DFE2818F0BD0000B7
:209200000304200000B528225043444A1018C2688A4201D3806800BD002000BD10B50400CA
:20922000282060433D4A1018826852188260C268511AC160C168002902D0C079002808D04B
:20924000200000F0E1F9200052490968896A00F05DFF10BDF1B582B00F0016006846007AC7
:20926000282148432D490818019000906846007A002808D127480268100048D031003800D0
:2092800000F07AFE43E000984269100003D03100380000F071FE009C08342068002827D0D6
:2092A0000099C9688E4201D2350001E00099CD68002D1DD02A00390000F0F6FE761B7F19D3
:2092C00001982168491921606168491B61606168002902D0C07900280AD06846007A00F084
:2092E00093F96846007A0C490968896A00F00EFF002E0CD03200390000981830FFF7A8FE13
:209300006846007A04490968896A00F0FFFE03B0F0BDC046180420001C04200084032000FE
:20932000F0B5040028206043A1490D18194E002C08D06879000602D4FF2000F07FF9307932
:20934000002808D0A968002923D02F88E868B84207D2EF6805E0287D00281AD10120287554
:20936000F0E73A00200033685B6B00F02DF9E868C01BE860A868C019A860E868002808D190
:2093800029888F4204D1A979002901D0A871F0BDA860F0BD1C042000F0B50400282060430B
:2093A00083490D18834E0027002C03D03079002800D12F75A868002805D02000FFF7B0FFAD
:2093C000307900281CD03079002803D1E868002800D1AF71A868002804D120003168896B08
:2093E00000F094FE002C09D0A868002808D1A879002805D1200000F007F9F0BD00F00EFDFE
:20940000F0BD000000B528224243694B9A181174684A1268126A00F0AFFD00BD6549086019
:2094200070470000F0B504000D0016001F001022002100F093FE6560A660E7602E480168C5
:209440000A0000E01268002A03D0A242FAD10120F0BD216004600020F0BD000030B50C4C3F
:20946000E0790025E570FFF777FD0120074902E00D70401C283122789042F9DBE079102160
:2094800001400820084300F013F830BDBC032000FC032000174800787047000015480178CE
:2094A0000120084304E0000012480178FE20084030B5354CE17981421BD0E0710E480568A1
:2094C000002D08D06968080002D0A86800F01EFE2D68002DF6D1E07980070AD5012504E06E
:2094E00000F054F86D1C2D062D0E280021788842F6D330BD030420002804200028214843B1
:209500002B490818006A704710B50400002A06D080208000844213D2022000F08FF8402CFD
:2095200001D3402010BD202C01D3202010BD102C01D3102010BD082C01D3082010BD0020D3
:2095400010BD000000B51B480068806900F0DCFD01000220084000BD00B516480068806980
:2095600000F0D2FD01000120084000BD10B506484478611C41700906090E022902D30720BB
:2095800000F05CF8200010BDFC03200000B528214143074A511800220A748A600A624A629D
:2095A0004B791B0600D50A7500F02EF800BD0000840320001C04200028225043014A101868
:2095C00041617047840320001847000030B51A4C03252000FEF7FAFB08346D1EF9D130BD31
:2095E00000B508484178491E4170090601D1FEF7E7F900BD00B5FEF7EDF902484178491C2A
:20960000417000BD6003200000B5C0000A490818FEF7E2FB00BD000000B5C00006490818FE
:20962000FEF72AFC00BD000000B5491CC000024A1018FEF739FC00BD2C04200000B50028F0
:2096400000D0FEE700BD000000B5026843689A4205D2836899540168491C016000BD042033
:20966000FFF7ECFF00BD000030B504000D000906090EFFF7E9FF290A2000FFF7E5FF30BD38
:20968000F0B585B0002000906E4802902820019009216846FFF7D8FF02216846FFF7D4FFE0
:2096A00000216846FFF7E0FF654801786846FFF7CBFF01216846FFF7C7FF00216846FFF721
:2096C000C3FFC0216846FFF7BFFF32216846FFF7BBFF0024594802E0641C04981430049039
:2096E00057480078844200DB9DE052480268002A04D069462000526800F03EFC0498039051
:20970000008840080025002804D0C10700D56D1C4008FAD109216846FFF796FF04216846E9
:20972000FFF792FF2106090E6846FFF78DFF00216846FFF789FF2906090E6846FFF784FF7A
:20974000039881786846FFF77FFF0398C1786846FFF77AFF039801796846FFF775FF002114
:209760006846FFF771FF03988168080002D0684600F0CCFC0125304E07E001273906090E08
:209780006846FFF761FF6D1C2836A34800788542A2DA039800880121A9400842F3D00721D5
:2097A0006846FFF751FF05216846FFF74DFF71796846FFF749FF31796846FFF745FFFFF741
:2097C000CBFE002804D13088412801D34020308031886846FFF748FF2820290041438F484E
:2097E00040180179012918D00329C6D14788FFF7B3FE002809D180204000874201D3FF27A7
:20980000BCE7002FBAD10827B8E7112F01D31027B4E7002FB2D10427B0E74788112FF6D2EC
:20982000002FABD1A9E77E4800990170054805B0F0BDC04624042000AC0320000404200029
:20984000FD03200044042000F0B585B000200090A24802902820019009216846FFF7F4FEE1
:2098600007216846FFF7F0FE00216846FFF7FCFE684801786846FFF7E7FE01216846FFF7F7
:20988000E3FE00216846FFF7DFFEC0216846FFF7DBFE32216846FFF7D7FE00245C4802E071
:2098A000641C0498143004905A480078844200DBA3E004980390008840080025002804D056
:2098C000C10700D56D1C4008FAD109216846FFF7BBFE04216846FFF7B7FE2106090E68465E
:2098E000FFF7B2FE00216846FFF7AEFE2906090E6846FFF7A9FE039881786846FFF7A4FEE6
:209900000398C1786846FFF79FFE039801796846FFF79AFE00216846FFF796FE0398816804
:20992000080002D0684600F0F1FB0126364D07E001273906090E6846FFF786FE761C28359D
:20994000354800788642ABDA039800880121B1400842F3D007216846FFF776FE052168466E
:20996000FFF772FE69786846FFF76EFE29786846FFF76AFEFFF7F0FD00280BD13006000EB8
:2099800022490968496900F0C1FB012229780004000C03E000222978281F0088FFF7B4FD9D
:2099A00001000904090C6846FFF75EFE3000282148431A4908180179012918D00329B7D1BD
:2099C0004788FFF7C9FD002809D180204000874201D3FF27ADE7002FABD10827A9E7112F19
:2099E00001D31027A5E7002FA3D10427A1E74788112FF6D2002F9CD19AE70948009901702B
:209A0000364805B0F0BDC046B00320001C04200004042000FD032000FC032000840320003F
:209A200046042000F0B584B028262C4D002700280FD100970295019604216846FFF704FE5D
:209A400003216846FFF700FE22496846FFF70CFE3DE0012806D0022808D0032809D0EE28EF
:209A60000BD00DE0FDF72AFE040007E0FDF72CFEFAE7FDF72FFE040000E017A4002C01D15A
:209A8000002025E022000020511C01E0401C491C13000A001B78002BF8D1039000970295EB
:209AA00001964100891C0906090E6846FFF7CCFD03216846FFF7C8FD0398002807D0060069
:209AC00021786846FFF7D0FD641C761EF8D1280004B0F0BD090400000000000044042000A1
:209AE000F0B584B00100002700263000CA7912028B79134303937A4C544DCA78012A09D01B
:209B0000022A4ED0032A4FD0062A51D0072A00D181E087E0009702952820019012216846AC
:209B2000FFF792FD01216846FFF78EFD802189006846FFF799FD21796846FFF785FD617951
:209B40006846FFF781FDA1796846FFF77DFD8E4801880906090E6846FFF776FDFDF7A4FD7A
:209B600001006846FFF780FDFDF7A4FD01006846FFF77AFD802149006846FFF775FD0121F0
:209B80006846FFF761FD02216846FFF75DFD03216846FFF759FD01216846FFF755FD280044
:209BA00040E0FFF76DFD3CE08878FFF73BFF39E0FFF7C8FC002837D00097029528200190D0
:209BC0000A216846FFF740FD06216846FFF73CFD802189006846FFF747FD21796846FFF725
:209BE00033FD61796846FFF72FFDA1796846FFF72BFD654801880906090E6846FFF724FD84
:209C000001216846FFF720FD00216846FFF71CFD2800AE7806E0FFF795FC002804D0FFF7D6
:209C200013FE8678002804D1206A406A00F06CFA0AE0002E00D1067803998E4200D30E00DA
:209C400001223100FFF746FA04B0F0BD4404200070B581B0224A146A8178C3781B020B43D2
:209C600005D18179C3791B020B43022B03D0606A00F04AFA31E0D1794907F8D50179037802
:209C80000320184000256E46D279920709D4012802D9801E02D020E0358019E00029FBD099
:209CA000E5E7002804D0012804D0022804D00EE001200BE035700AE00800FFF725F9FF2815
:209CC000D5D02821484330490818007C30707570002202216846FFF7FDF901B070BD0000B4
:209CE000FC032000F0B581B002000C004A4D286A00902606360E9078D1780902014304D1C3
:209D00009079D1790902014305D00098406A00F0FBF901B0F0BDE8794007F6D510791278C2
:209D200003211140EA79920718D4002904D00129EBD0022906D0ECE7012200210120FFF7B5
:209D4000C9F9E6E7FFF7E0F80700DED10E48002C02D001210174EFE70021FBE70029EBD048
:209D60000229D2D1FFF7D0F80700FF2FCDD03100FFF748FB002EDFD1286AC16B0800DBD0CC
:209D8000380000F0C3F9D7E78403200070B581B0694680780870204C206A0500097801295F
:209DA00027D1012200210120FFF794F9E17902200843FFF77DFB01260FE00021FFF722FB44
:209DC000206AC16B080002D0300000F09FF93000FFF7DCFB761C3606360E30002178884299
:209DE000EBD32A6C100015D06946002000F0C4F810E069460978002909D101220120FFF742
:209E000069F9E179FD200840FFF752FBE9E7406A00F07AF901B070BDFC03200030B5554C7E
:209E2000E078000615D5E0784006400EE070E5782800216AC96900F069F9002DE17904D0AF
:209E400004200843FFF734FB30BDFB200840FFF72FFB30BDF0B582B00400464F7878019020
:209E6000002600280ED03D0008352969080004D0200000F04BF900287AD0761C1435019894
:209E80008642F2D3396A0D0020786022024002D0202A5AD057E0A078062263780B2B52D831
:209EA00001A6F65CB744C0460C149E1E9E22369E3E525A802000FFF7CBFE59E00021200075
:209EC000FFF710FF54E00121F9E70400012200210120FFF7FFF880202043F87048E020003E
:209EE000FFF7FEFD44E0FFF731F869460870002201216846FFF7EEF83AE02000FFF746FFC4
:209F000036E0002802D1A079012803D0486A00F0FBF82DE0F8790240062AF7D168460021FF
:209F2000017000220121E5E72079FB791A40062A03D0486A00F0E8F81AE0496A7A78824251
:209F400000F0E4F814E0686AE1E7002601980028F9D0083704E0761C143701988642F2D2D2
:209F6000F9680800F7D0200000F0D0F80028F2D102B0F0BDFC032000104700000102000A0C
:209F800008430004000C7047F6B581B004001D0007210A4209D1D60832000199200000F0AA
:209FA00083F8A4196D1EF7D124E00020019900910299621C02E0641C0839521C009B1B786F
:209FC000009E761C009600280AD083402678FF278740BE431F00374327701B0A137000E0B2
:209FE00023700829E7DA4018C10864184007400F6D1EDBD103B0F0BD00B5884200DB0800B0
:20A0000000BD000002681170521C02607047000002681170090A5170921C0260704700008B
:20A0200002681170090A5170090A9170090AD170121D0260704700000170090A4170801CE0
:20A04000090A0170090A41707047000000B50029017803D009024078084300BD4078000252
:20A06000084300BD01780906427812040A43817809021143C078084370470000017842786E
:20A0800012020A43817809041143C078000608437047000000B5002902D0FFF7E3FF00BD80
:20A0A000FFF7ECFF00BD0000004B1847240F200000B5FDF78FFC0C484178491C4170F7F0C7
:20A0C00001F8FEF7C7F8FDF7E1FDFEF775F8074801B4074B074A64210748FDF70DFE00F035
:20A0E0000DF801B000BDC0466003200068090000F4042000197410005C0E2000004B18470A
:20A10000907F100000B5FEE7004700000847000000B581B000F02EF801B000BD10B5002A97
:20A120000DD003780C78A34205D002D20020C04310BD012010BD401C491C521EF1D10020C4
:20A1400010BD000010B50300002A05D00C78491C1C705B1C521EF9D110BD000000B50906B4
:20A16000090E0300002A03D019705B1C521EFBD100BD0000014CA6462047000005A1100079
:20A180007847C0460C002DE900C0A0E3060000EA7847C0460C002DE941C0B0E10010612299
:20A1A0008CC0A0E140C03CE0000060220120B0E13100000A0030A0E3200851E10118A091F0
:20A1C000200451E10114A091A00051E12000008A200151E11C00008AA00151E11700008AFA
:20A1E000200251E11200008AA00251E10D00008A200351E10800008AA00351E10300008ABB
:20A20000810350E1810340200330A3E0010350E1010340200330A3E0810250E18102402009
:20A220000330A3E0010250E1010240200330A3E0810150E1810140200330A3E0010150E19D
:20A24000010140200330A3E0810050E1810040200330A3E0010050E1010040200330A3E054
:20A26000020051E12114A081E4FFFF8A0310A0E18C3FB0E100106122000060420C00BDE812
:20A280001EFF2FE17847C046F0412DE90140A0E10280A0E10350A0E1006090E574709FE5AF
:20A2A00074009FE50000D0E5000050E30C00000A040094E4D50100EBA86186E0078008E28B
:20A2C0000820A0E10010A0E10600A0E1DD0100EB040097E5088080E0015055E2F3FFFF1AF9
:20A2E000090000EA041094E4A86186E0078008E20820A0E10600A0E1D20100EB040097E591
:20A30000088080E0015055E2F5FFFF1A0400A0E1F041BDE81EFF2FE118012000D20020000D
:20A32000030052E33D00009A03C010E20800000A0130D1E402005CE30C2082E001C0D1946C
:20A340000130C0E40130D13401C0C094042042E20130C034033011E21D00000A042052E2CB
:20A360002E00003A03C031E7020053E30800000A0F00008A2C34A0E104C0B1E5042052E224
:20A380000C3C83E1043080E4F9FFFF2A011081E2220000EA2C38A0E104C0B1E5042052E241
:20A3A0000C3883E1043080E4F9FFFF2A021081E21A0000EA2C3CA0E104C0B1E5042052E228
:20A3C0000C3483E1043080E4F9FFFF2A031081E2120000EA202052E210402DE90500003A95
:20A3E0001850B1E81850A0E81850B1E81850A0E8202052E2F9FFFF2A02CEB0E11850B12844
:20A400001850A0281800B1481800A04802CFB0E11040BDE804309124043080241EFF2F0196
:20A42000822FB0E10120D1440130D12401C0D1240120C0440130C02401C0C0241EFF2FE1BC
:20A44000F0B581B004000D001600184800681F2188438027202100911549884202D015495B
:20A46000884202D180374020009000F039F89720C0432100009A2B6823602D1D241D521EF1
:20A48000F9D1802F00D149009B23DB430A4A0A400A49114319600168C907FCD5F61B012E45
:20A4A000E7DA06F7B9FC01B0F0BDC04640F2FFFF40090D2740095B2700FF03000100005AF0
:20A4C00000B59720C0430168C90606D49B21C943024A0A600168C907FCD500BD0F00005A4D
:20A4E000004B1847D87910007847C046F0072DE91CC09DE520409DE5EF50E0E3C05FC5E376
:20A50000496FA0E3006085E5FB50E0E3B05EC5E3706AA0E3006085E58060A0E3006082E521
:20A52000B4609FE52C7096E5047082E5306096E5306082E50160A0E3006082E5807CA0E365
:20A54000007083E5046083E50770A0E31C7083E50280A0E3188083E5408FA0E3008083E52A
:20A560000180D0E4248083E58088A0E30C9085E2008089E5309085E3008089E52CA085E2D5
:20A5800000808AE5008089E500808AE5008089E500808AE5109085E3008089E52180A0E3F8
:20A5A000108083E5147083E5006083E5606CA0E3006085E5081182E5080183E500C183E5BC
:20A5C000010044E20C0183E5044183E5FA0087E2200183E5F007BDE81EFF2FE13802200023
:20A5E0000C214843401EFDD170470000F04F2DE968739FE540BCA0E303E0A0E10140D0E434
:20A600000150D1E480CBA0E30880A0E3080053E30380A041083043E000A0A0E3A440B0E1C6
:20A6200080AB8A23A550B0E180AD8A2338A087E501C05CE21900000A3CA097E540001AE3E7
:20A64000FAFFFF1A30B087E501C05CE21300000A3CA097E540001AE3FAFFFF0AAAA6B0E108
:20A660006660A0E1018058E2EAFFFF1A266CB0E10160C2E4000053E3DFFFFF1A07301EE248
:20A68000083063123663A011016042150000A0E380ADA0E334A087E5F04FBDE81EFF2FE187
:20A6A00030B087E50100A0E3F8FFFFEAAD4B1847AD4B1847F0B5FFF7F9FFA94F0024402528
:20A6C00001263603BC63C046F86BF96BFA6BFB6BFC6B2C4204D0761EFAD10020401E10E0ED
:20A6E000284220D0294220D02A4220D02B4220D001210903881B0921484315214843C830AD
:20A7000073300124A403BC6301263603761E07D0FC6B2C42FAD0041CFFF7CAFF201CF0BD79
:20A720000020401EF7E70020EBE77E20E9E7BD20E7E7FC20E5E70000F04F2DE924409DE58F
:20A74000020000EAF04F2DE91C429FE5004094E508929FE580ADA0E340BCA0E303E0A0E16C
:20A76000000054E32300000A0150D0E40160D1E40880A0E3080053E30380A041083043E052
:20A7800010C0A0E3A550B0E134C0892530C08935A660B0E130A0892534A0893530B089E59B
:20A7A00004C0A0E101C05CE2FDFFFF1A34B089E504C0A0E101C05CE2FDFFFF1A3CC099E51B
:20A7C000ACC5B0E16770A0E1018058E2EBFFFF1A277CB0E10170C2E4000053E3E1FFFF1AE7
:20A7E00007301EE2083063123773A01101704215F04FBDE81EFF2FE110C0A0E30150D0E4E9
:20A800000160D1E40880A0E3080053E30380A041083043E0080058E33600001A000055E34F
:20A820001C00000AFF0055E33200001A34C089E5A660B0E130A0892534A0893530B089E518
:20A8400034B089E5A660B0E130A0892534A0893530B089E534B089E5A660B0E130A089254A
:20A8600034A0893530B089E534B089E5A660B0E130A0892534A0893530B089E534B089E55F
:20A88000048058E2E9FFFF1A012082E2000053E3D9FFFF1AD1FFFFEA30C089E530B089E5E8
:20A8A00034B089E53C4099E5A445B0E16770A0E130B089E534B089E53C4099E5A445B0E166
:20A8C0006770A0E130B089E534B089E53C4099E5A445B0E16770A0E130B089E534B089E514
:20A8E0003C4099E5A445B0E16770A0E1048058E2E9FFFF1A140000EAA550B0E10900002A16
:20A90000A660B0E130C0893530B089E534B089E53C4099E5A445B0E16770A0E1018058E2CB
:20A92000F4FFFF1A080000EA34C089E5A660B0E130A0892534A0893530B089E534B089E570
:20A940006770A0E1018058E2EAFFFF1A277CB0E10170C2E4000053E3A7FFFF1A9FFFFFEA1B
:20A9600000F4FFFFD8791000C47910003402200010B510480068104C2178491C2170617898
:20A98000491C617000F01EF80C48002101606078401E60702078012805D109480078002817
:20A9A00001D000F011F82078401E207010BC01BC0047C04600F1FFFF6003200030F1FFFFE0
:20A9C0007F0E200000470000004B1847C47F10000F502DE900004FE101002DE993F021E343
:20A9E00000402DE91C009FE50FE0A0E110FF2FE10040BDE892F021E30200BDE801F06FE17F
:20AA00000F50BDE804F05EE2751520007847C04628109FE5202CD1E70034A0E1233CD1E703
:20AA2000032482E10038A0E1233CD1E7032882E1000CA0E1200CD1E7000C82E11EFF2FE121
:20AA400078AD10007847C046033000E2832182E00300C0E3000052E30A00000A0130A0E33E
:20AA60001332A0E1013043E200C090E50CC003E011C28CE104C080E400C090E50330CCE159
:20AA8000202062E2311283E1001080E51EFF2FE17847C04630002DE900C0A0E3A10180E099
:20AAA000071011E20900000A084041E2033084E001C0D2E40040D0E5FF50A0E31551E0E112
:20AAC000044005E01C51A0E1044085E10140C0E4081061E2080053E32300003AA341A0E175
:20AAE000040054E31600003A0150D2E405C48CE13C51A0E10150C0E40150D2E40554A0E1AA
:20AB00002CC485E13C51A0E10150C0E40150D2E40554A0E12CC485E13C51A0E10150C0E4A2
:20AB20000150D2E40554A0E12CC485E13C51A0E10150C0E42CC4A0E1044044E2040054E3C5
:20AB4000E8FFFF2A000054E30600000A0150D2E405C48CE13C51A0E10150C0E42CC4A0E1ED
:20AB6000014054E2F8FFFF1A073003E2000053E30700000A0020D2E502248CE13211A0E1BD
:20AB80000120A0E31223A0E1012042E2011002E00010C0E53000BDE81EFF2FE1EC0D000073
:20ABA0009C0020009C00200018090000880E200084A210005500000044002000CCAB1000D0
:20ABC00018090000880E200084A210000100000004000000B80B000031323334353600006B
:20ABE00000000000FCAC100004AD100000400000000000000000000000000000000000009C
:20AC000000100000000000008025000000010800000E4000000E4000000940006613010116
:20AC200030FFFFFFFF00000000E00000FFE0FFFFFFFF000081C0030000000000BD0000002C
:20AC4000000000009F00000000000000B700000000000000A5000000000000008D0000006C
:20AC600000000000FFFFFFFFFFFFFF9EE7FFFFFFFFFFFFFFB6EDFFFFFFFFFFFFFF0000A51C
:20AC80000000000000000000FFFFFFFFFFFFFFFFFFFFFFFFFFFFFFFFFFFFFFFFFFFFFFFFCC
:20ACA000FFFFFFFF00000000F00000004941524B53000000BF7BFFB98038010080380100CA
:20ACC000803801008038010080380100803801008038010080380100808D5B0001000000B5
:20ACE000FFFF0000000000000000000069751000A5751000BD751000BD7410005345474795
:20AD0000455200004A2D4C696E6B00006D791000757910009977100015791000517910000B
:20AD2000A9771000A9781000D5781000BD7710005D781000A58C1000E58C10005D8B100072
:20AD40009D8C1000558B1000198D1000298D1000E58A1000498C1000BD8A1000098B1000EF
:20AD6000198B1000B18B1000298B1000A18C10002D8D1000618D1000008040C020A060E08A
:20AD8000109050D030B070F0088848C828A868E8189858D838B878F8048444C424A464E413
:20ADA000149454D434B474F40C8C4CCC2CAC6CEC1C9C5CDC3CBC7CFC028242C222A262E2A3
:20ADC000129252D232B272F20A8A4ACA2AAA6AEA1A9A5ADA3ABA7AFA068646C626A666E693
:20ADE000169656D636B676F60E8E4ECE2EAE6EEE1E9E5EDE3EBE7EFE018141C121A161E13B
:20AE0000119151D131B171F1098949C929A969E9199959D939B979F9058545C525A565E572
:20AE2000159555D535B575F50D8D4DCD2DAD6DED1D9D5DDD3DBD7DFD038343C323A363E302
:20AE4000139353D333B373F30B8B4BCB2BAB6BEB1B9B5BDB3BBB7BFB078747C727A767E7F2
:20AE6000179757D737B777F70F8F4FCF2FAF6FEF1F9F5FDF3FBF7FFFFFFF0000000000002C
:20AE80000000000000000000000000000000000000000000000000000000000000000000B2
:20AEA000000000000000000000000000000000000000000000000000000000000000000092
:20AEC000000000000000000000000000000000000000000000000000000000000000000072
:20AEE000000000000000000000000000000000000000000000000000000000000000000052
:20FB00007777772E7365676765722E636F6D00436F70797269676874202863292032303029
:20FB200033202D203230303920534547474552204D6963726F636F6E74726F6C6C65722EF1
:20FB4000204D6179206265207573656420696E206F726967696E616C204A2D4C696E6B73A2
:20FB600020616E642070726F6475637473206D616E75666163747572656420756E64657241
:20FB8000206C6963656E7365206F6E6C792E00000000000000000000000000000000000052
:20FBA000000000000000000000000000000000000000000000000000000000000000000045
:20FBC000000000000000000000000000000000000000000000000000000000000000000025
:20FBE0000000000000000000000000000000000000000000000000000000000000003F4284
:20FC0000FFFFFFFFFFFFFFFFFFFFFFFFFFFFFFFFFFFFFFFFFFFFFFFFFFFFFFFFFFFFFFFF04
:20FC2000FFFFFFFFFFFFFFFFFFFFFFFFFFFFFFFFFFFFFFFFFFFFFFFFFFFFFFFFFFFFFFFFE4
:20FC4000FFFFFFFFFFFFFFFFFFFFFFFFFFFFFFFFFFFFFFFFFFFFFFFFFFFFFFFFFFFFFFFFC4
:20FC6000FFFFFFFFFFFFFFFFFFFFFFFFFFFFFFFFFFFFFFFFFFFFFFFFFFFFFFFFFFFFFFFFA4
:20FC8000FFFFFFFFFFFFFFFFFFFFFFFFFFFFFFFFFFFFFFFFFFFFFFFFFFFFFFFFFFFFFFFF84
:20FCA000FFFFFFFFFFFFFFFFFFFFFFFFFFFFFFFFFFFFFFFFFFFFFFFFFFFFFFFFFFFFFFFF64
:20FCC000FFFFFFFFFFFFFFFFFFFFFFFFFFFFFFFFFFFFFFFFFFFFFFFFFFFFFFFFFFFFFFFF44
:20FCE000FFFFFFFFFFFFFFFFFFFFFFFFFFFFFFFFFFFFFFFFFFFFFFFFFFFFFFFFFFFFFFFF24
:20FD0000FFFFFFFFFFFFFFFFFFFFFFFFFFFFFFFFFFFFFFFFFFFFFFFFFFFFFFFFFFFFFFFF03
:20FD2000FFFFFFFFFFFFFFFFFFFFFFFFFFFFFFFFFFFFFFFFFFFFFFFFFFFFFFFFFFFFFFFFE3
:20FD4000FFFFFFFFFFFFFFFFFFFFFFFFFFFFFFFFFFFFFFFFFFFFFFFFFFFFFFFFFFFFFFFFC3
:20FD6000FFFFFFFFFFFFFFFFFFFFFFFFFFFFFFFFFFFFFFFFFFFFFFFFFFFFFFFFFFFFFFFFA3
:20FD8000FFFFFFFFFFFFFFFFFFFFFFFFFFFFFFFFFFFFFFFFFFFFFFFFFFFFFFFFFFFFFFFF83
:20FDA000FFFFFFFFFFFFFFFFFFFFFFFFFFFFFFFFFFFFFFFFFFFFFFFFFFFFFFFFFFFFFFFF63
:20FDC000FFFFFFFFFFFFFFFFFFFFFFFFFFFFFFFFFFFFFFFFFFFFFFFFFFFFFFFFFFFFFFFF43
:20FDE000FFFFFFFFFFFFFFFFFFFFFFFFFFFFFFFFFFFFFFFFFFFFFFFFFFFFFFFFFFFFFFFF23
:20FE0000FFFFFFFFFFFFFFFFFFFFFFFFFFFFFFFFFFFFFFFFFFFFFFFFFFFFFFFFFFFFFFFF02
:20FE2000FFFFFFFFFFFFFFFFFFFFFFFFFFFFFFFFFFFFFFFFFFFFFFFFFFFFFFFFFFFFFFFFE2
:20FE4000FFFFFFFFFFFFFFFFFFFFFFFFFFFFFFFFFFFFFFFFFFFFFFFFFFFFFFFFFFFFFFFFC2
:20FE6000FFFFFFFFFFFFFFFFFFFFFFFFFFFFFFFFFFFFFFFFFFFFFFFFFFFFFFFFFFFFFFFFA2
:20FE8000FFFFFFFFFFFFFFFFFFFFFFFFFFFFFFFFFFFFFFFFFFFFFFFFFFFFFFFFFFFFFFFF82
:20FEA000FFFFFFFFFFFFFFFFFFFFFFFFFFFFFFFFFFFFFFFFFFFFFFFFFFFFFFFFFFFFFFFF62
:20FEC000FFFFFFFFFFFFFFFFFFFFFFFFFFFFFFFFFFFFFFFFFFFFFFFFFFFFFFFFFFFFFFFF42
:20FEE000FFFFFFFFFFFFFFFFFFFFFFFFFFFFFFFFFFFFFFFFFFFFFFFFFFFFFFFFFFFFFFFF22
:20FF0000FFFFFFFFFFFFFFFFFFFFFFFFFFFFFFFFFFFFFFFFFFFFFFFFFFFFFFFFFFFFFFFF01
:020000040010EA
:20FF20005244492C466C617368444C2C466C61736842502C4A466C6173682C474442467574
:020000040010EA
:20FF40006C6C00FF802020207BE2B7DDC407C20AFFFFFFFFFFFFFFFFFFFFFFFFFFFFFFFF72
:020000040010EA
:20FF6000FFFFFFFFFFFFFFFFFFFFFFFFFFFFFFFFFFFFFFFFFFFFFFFFFFFFFFFFFFFFFFFFA1
:020000040010EA
:20FF8000FFFFFFFFFFFFFFFFFFFFFFFFFFFFFFFFFFFFFFFFFFFFFFFFFFFFFFFFFFFFFFFF81
:020000040010EA
:20FFA000FFFFFFFFFFFFFFFFFFFFFFFFFFFFFFFFFFFFFFFFFFFFFFFFFFFFFFFFFFFFFFFF61
:020000040010EA
:20FFC000FFFFFFFFFFFFFFFFFFFFFFFFFFFFFFFFFFFFFFFFFFFFFFFFFFFFFFFFFFFFFFFF41
:020000040010EA
:20FFE000FFFFFFFFFFFFFFFFFFFFFFFFFFFFFFFFFFFFFFFFFFFFFFFFFFFFFFFFFFFFFFFF21
:00000001FF
